:1000000000800020BD010000515B00001D5B00006E
:100010001D5B00001D5B00001D5B00001D5B000000
:100020001D5B00001D5B00001D5B0000515B0000BC
:10003000515B00001D5B0000515B00000D5B000088
:10004000515B0000515B0000515B0000515B000000
:10005000515B0000515B0000515B0000515B0000F0
:10006000515B0000515B0000515B0000515B0000E0
:10007000515B0000515B0000515B0000515B0000D0
:10008000515B0000515B0000515B0000515B0000C0
:10009000515B0000515B0000515B0000515B0000B0
:1000A000515B0000515B0000515B0000515B0000A0
:1000B000515B0000515B0000515B0000515B000090
:1000C000515B0000515B0000515B0000515B000080
:1000D000515B0000515B0000515B0000515B000070
:1000E000515B0000515B0000515B0000515B000060
:1000F000515B0000CD670000515B0000916D000076
:10010000515B00006D720000515B0000515B00000C
:10011000515B0000515B0000515B0000515B00002F
:10012000515B000015080000450B0000515B00000A
:10013000515B0000515B0000515B0000515B00000F
:10014000515B0000515B0000515B0000515B0000FF
:10015000A9810000C1810000D9810000F181000067
:10016000515B000075750000515B0000515B0000A1
:10017000515B0000515B0000515B0000515B0000CF
:10018000515B0000515B0000515B0000095300000F
:10019000515B0000515B0000515B0000515B0000AF
:1001A000515B0000515B0000515B0000515B00009F
:1001B000515B0000515B0000515B0000564B4CF25C
:1001C000205210B51A804DF628121A8000BF00BFC9
:1001D00005F0C2FC514B4FF010621A60504A9A6011
:1001E000504ADA60A3F53043203B1A6812F480725B
:1001F00004D14D490A604FF4A8521A604B4B1A784B
:10020000110703D51A7842F008021A70484B2A22C7
:100210001A700023474A48499818884204D247492F
:10022000595899500433F5E7454A464B9A424FF0E6
:10023000000302D242F8043BF7E74349434A5958C6
:1002400099500433B3F5DE7FF7D1414B802103F899
:10025000011B40498B42F9D13F4B1A603F4B0A22A8
:100260001A70A3F5805324225A70A0221A709A792A
:100270009207FCD59A79D406FCD4394B9A7902F0CE
:100280000C02082AF9D103221A7140225A719A7974
:100290009006FCD5324B9A795106FBD5314A32494A
:1002A00011600221516020221A702D4B9B7903F0BE
:1002B0000C030C2BF9D12D4B2D4A1A602D4B2E4AD5
:1002C0001A6000225A60072243F8042C2B4AC3F814
:1002D0000C2D62B605F0D6FF134B1B68DA0705D567
:1002E000274805F0F3FD274B274A1A60274B1B7858
:1002F0005B0609D5234C244A2368934204D1204845
:1003000005F0E4FD0023236008F002FD05F02AFC5F
:1003100008F02BF8FEE700BF0E20054030800440B7
:10032000823F04000100002B14D0034002D007409C
:1003300000E007406087FF1F8088FF1F64C1000046
:100340008088FF1F0892FF1F000000000082FF1F2F
:1003500000E400E05FE400E008ED00E0005006404B
:100360000040064044800440000003010480044033
:10037000C010050014E000E0FF760100000020201E
:1003800000DD68501CE00340A5C3945A00F007400C
:10039000FFFFFFFFFFFFFFFFFFFFFFFFFFFFFFFF6D
:1003A000FFFFFFFFFFFFFFFFFFFFFFFFFFFFFFFF5D
:1003B000FFFFFFFFFFFFFFFFFFFFFFFFFFFFFFFF4D
:1003C000FFFFFFFFFFFFFFFFFFFFFFFFFFFFFFFF3D
:1003D000FFFFFFFFFFFFFFFFFFFFFFFFFFFFFFFF2D
:1003E000FFFFFFFFFFFFFFFFFFFFFFFFFFFFFFFF1D
:1003F000FFFFFFFFFFFFFFFFFFFFFFFFFFFFFFFF0D
:10040000FFFFFFFFFFFFFFFFFFFFFFFFFEFFFFFFFD
:1004100010B5054C237833B9044B13B10448AFF33E
:1004200000800123237010BD8088FF1F00000000A2
:1004300064C1000008B5064B1BB106480649AFF37E
:1004400000800648036813B1054B03B1984708BD07
:100450000000000064C100008488FF1F8088FF1F27
:10046000000000002DE9F04101210D2005F0D6FD2E
:100470006D4B6E4C6E4E20221A604FF4887007F060
:100480007CFF054602F03AFC2846256002F0C3FBDB
:10049000FE2811D140F2DC5005F0DEFE902007F07E
:1004A0006CFF644904464FF4E13201F0A5F8346072
:1004B000306802F073F9FBE723685F4993F8AA00FC
:1004C00005F014FD5D4B4FF496721A605C4BC02230
:1004D0001A602368012193F8AA0005F09FFD2368A4
:1004E000402193F8AA0005F0B5FD0C2005F0ECF8CA
:1004F000082005F013F940F2DC5005F0ADFE20684D
:1005000002F04BFB430803F1376303F5D833B3FB29
:10051000F0F005F005FF206802F061FB20B12368D0
:1005200093F8A80005F0A8FF206802F062FB4308DA
:1005300003F1376303F5D833B3FBF0F006F0DAF9D3
:10054000206802F05FFB430803F1B76303F55843EB
:10055000B3FBF0F006F0B0FC206802F04AFB054661
:100560005C2007F00AFF2A463649374D074603F05C
:10057000AFFE20682F6002F010FB80466C2007F071
:10058000FCFE42463149074603F05EFA304B5820E4
:100590001F6007F0F2FE074600F096FC2D4B2E4937
:1005A0001F60384600F0FCFD902007F0E6FE214970
:1005B0004FF4E132074601F01FF82068376002F07F
:1005C00021FB0746902007F0D8FE3A46224906460E
:1005D00001F012F8214B28681E6003F0ADFF286877
:1005E0001F4E03681B6A98473768286807F2FD2783
:1005F00003F0A6FE3368BB4204D2286803681B6A76
:100600009847F7E760210B4620680A4602F089FA0E
:1006100000F0DAF823681B7E23B10120BDE8F04129
:1006200004F074BDBDE8F08184F00F40B888FF1F6E
:100630009C88FF1FD091FF1F0000A041A888FF1FCA
:10064000A088FF1F9891FF1FC088FF1F8891FF1F80
:10065000B488FF1FB088FF1FA891FF1FBC88FF1F31
:10066000D489FF1F1C4B1A684FF6E85101328A42A9
:1006700070B51A601D462EDD184C2368D3F8B400FF
:1006800004F0F2F923680C2690FBF6F6986804F063
:10069000E1F9B0F5967F05DDB0F5167FA8BF4FF400
:1006A000167001E04FF496700D4A23681268A0F5A9
:1006B00096700A21414391FBF2F10A4A93F8AA008D
:1006C0001268514301F52071F6B291FBF6F105F085
:1006D000C1FC00232B6070BDAC88FF1FB888FF1FD2
:1006E000A888FF1FA088FF1F0F4B1A68002A08DA8E
:1006F0000E49086801280DD00120086020200C490F
:1007000007E007D00949086820B1002008600949BE
:100710002020086001324FF6E8518A42C8BF6FF0CE
:1007200031021A60704700BFA488FF1F6487FF1F53
:1007300084F00F4088F00F402DE9F0411D4F1E4D11
:100740003B681E4C93F8C430DFF878801C4E93B998
:10075000286802F023F8206802F020F8D8F800009A
:1007600003F0D0FB306803681B6A9847FFF77AFFF5
:10077000FFF7BAFFE2E7D8F8000010B103689B6802
:100780009847306810B103689B689847286810B193
:1007900003689B689847206810B103689B68984776
:1007A00000F02EF83B681B7E0BB104F01DFE00F03C
:1007B00059FAFCE7B888FF1F9C88FF1FBC88FF1F01
:1007C000C088FF1FB488FF1F08B5094B4FF00072A7
:1007D0001A604FF080621A60064B1B6893F8250080
:1007E000054B187005F034F8044B01221A7008BD4F
:1007F00004E100E0B888FF1FC488FF1FC688FF1F00
:10080000034B4FF000721A604FF080621A6070471D
:1008100084E100E070B5B24C23780F2B00F28781A1
:10082000DFE813F0210036004B00600075008A00FD
:100830009F00B400C900DE001D0134010101680100
:100840004A011000A74D287805F04AF8A64B1B680E
:10085000D3F8B420132101FB0200142690FBF6F21A
:10086000C3F8B420D8E09F4D287805F039F89E4BA6
:100870001B681A6B452101FB0200462690FBF6F22D
:100880001A6393F82500287004F0E2FF01234CE17D
:10089000944D287805F024F8934B1B685A6B45213A
:1008A00001FB0200462690FBF6F25A6393F82600FD
:1008B000287004F0CDFF022337E18A4D287805F037
:1008C0000FF8894B1B689A6B452101FB02004626F5
:1008D00090FBF6F29A6393F82700287004F0B8FFB3
:1008E000032322E17F4D287804F0FAFF7E4B1B683A
:1008F000DA6B452101FB0200462690FBF6F2DA6333
:1009000093F82800287004F0A3FF04230DE1754D2F
:10091000287804F0E5FF744B1B681A6C452101FB35
:100920000200462690FBF6F21A6493F8290028701C
:1009300004F08EFF0523F8E06A4D287804F0D0FF1C
:10094000694B1B685A6C452101FB0200462690FB4F
:10095000F6F25A6493F82A00287004F079FF06230F
:10096000E3E0604D287804F0BBFF5F4B1B689A6C96
:10097000452101FB0200462690FBF6F29A6493F8AB
:100980002B00287004F064FF0723CEE0554D287833
:1009900004F0A6FF544B1B68DA6C452101FB0200F2
:1009A000462690FBF6F2DA6493F82C00287004F0E7
:1009B0004FFF0823B9E04B4D287804F091FF4A4BD4
:1009C0001B681A6D452101FB0200462690FBF6F2DA
:1009D0001A6593F82D00287004F03AFF0923A4E06B
:1009E000404D287804F07CFF3F4B1B685A6D452131
:1009F00001FB0200462690FBF6F25A653B4A11784D
:100A0000092907D9987B28700021117004F020FF74
:100A10000C238AE00131117093F82400287004F04F
:100A200017FF002381E02F4D287804F059FF2E4B4B
:100A30001B681A69632101FB0200642690FBF6F231
:100A4000597B1A612A4A52F83120012182F880101C
:100A500093F89F00287004F0FBFE0A2365E0214D07
:100A6000287804F03DFF204B1B68D3F8A42002EB4C
:100A7000C20210440A2190FBF1F2C3F8A42093F8BB
:100A80009E00287004F0E4FE0B234EE0154D2878FC
:100A900004F026FF144B1B68D3F8A02002EBC2021F
:100AA00010440A2190FBF1F2C3F8A02018792870B5
:100AB00004F0CEFE0E2338E00A4D287804F010FF33
:100AC000094B1B689A68312101FB0200322690FB1A
:100AD000F6F29A60987B287004F0BAFE0D2324E0A9
:100AE000C688FF1FC488FF1FB888FF1FC588FF1F67
:100AF000E4BC0000104D287804F0F2FE0F4B1B6898
:100B00005A69632101FB0200642690FBF6F2597BCF
:100B10005A610B4A52F83120012182F8001193F8F2
:100B2000B000287004F094FE0F23237070BD0220E3
:100B3000BDE8704003F0A4BFC488FF1FB888FF1F42
:100B4000E4BC0000FFF766BEF8B5404D05F04AFF73
:100B50002F7807F001073E4C0021802320680A46C9
:100B600001F0DFFF2B7813F0010F264609D104F0C6
:100B700033FA2B78DA0706D4FFF7B6FDFFF772FDDC
:100B8000F7E7002F37D12B78DB0734D54FF4FA7015
:100B900005F062FB2F4B20681F6802F048F82E49D1
:100BA00003463A462D4807F023FC07F0A3F8002837
:100BB000FBD000210A2005F031FA206802F02CFB5E
:100BC000206802F028F8032802D1192005F044FB20
:100BD0000A20012105F022FA01210A2005F0FEF980
:100BE000192005F039FB1B4B0A20196804F0CEF9D7
:100BF0001B4B80221A602F7807F0010707F07AF864
:100C000060B107F035F8FF210446002230688023E8
:100C100001F087FFE0B204F025FAEFE704F0F8F9FD
:100C200070B104F005FA00210446FF2230688023E9
:100C300001F077FF09480268214612689047EDE706
:100C4000FFF710FDFFF750FD85E700BF8491FF1F00
:100C5000B888FF1FF891FF1FE49B0000D091FF1F91
:100C600088F00F402DE9F84F804F3B6893F8C4603F
:100C700016F0100F06F0040807D0B8F1000F01D0ED
:100C8000FFF762FF1B2003F0FBFE16F0020F784C0B
:100C9000784D0DD02268784B0AB9236001E0774A7D
:100CA00013602A7802230AB9724A00E0744A13706A
:100CB000B8F1000F0DD02268724B0AB96C4A00E0FF
:100CC0006E4A13602A7804230AB96A4A00E06C4A23
:100CD000137033070DD522686B4B0AB9644A00E0E4
:100CE000664A13602A7808230AB9624A00E0644A17
:100CF0001370F0070DD52268644B0AB95C4A00E016
:100D00005E4A13602A7801230AB95A4A00E05C4A15
:100D100013705F4E96F8008008F0010800218023D0
:100D200038680A4601F0FDFE2B78012B03D0544BA6
:100D30001B78012B3CD13378D9071FD42368534A41
:100D4000934208BF4D4B4C4A08BF1B68934202D1E7
:100D500005F05EFB0AE04B4A934202D105F042FEE9
:100D600004E0494A934201D106F012F93378DA07D8
:100D7000FCD54FF4FA7005F06FFA02E0B8F1000FFD
:100D800016D13378DB0713D52368404A934201D14B
:100D90003A4B1B68384A93424AD13E4B1868430885
:100DA00003F1376303F5D833B3FBF0F005F0B8FA7D
:100DB00096F8008008F001082068DFF8C09003680A
:100DC0009B689847A0B13868FF210022802301F07A
:100DD000A8FED9F80090D9F80030D3F800A0244B31
:100DE00018680368DB689847C1B24846D047E3E714
:100DF000D9F8000003689B689847A0B138680021C3
:100E0000FF22802301F08DFED4F800A0DAF8003034
:100E1000D3F800B0194B18680368DB689847C1B273
:100E20005046D847E4E7FFF71DFCFFF75DFC75E788
:100E3000144A93420BD1174B1868430803F13763E8
:100E400003F5D833B3FBF0F005F054FDB0E70E4ADC
:100E50009342ADD10F4B1868430803F1B76303F514
:100E60005843B3FBF0F006F027F8A1E7B888FF1F5E
:100E7000D088FF1FCC88FF1F8891FF1FC888FF1FE5
:100E8000CD88FF1F9891FF1FA891FF1FD091FF1FD2
:100E90008491FF1FF891FF1F38B5044608460D46A0
:100EA00008F07DF8236802465B682046294698478B
:100EB00038BD38B50446FFF7EFFF0546204607F07A
:100EC00081FA284438BDFFFF38B500250446057176
:100ED000457180F8545004491422063008F07EF819
:100EE0002565204638BD00BF959C000000797047FD
:100EF00090F85520044B53F83220012382F88030BB
:100F000003711846704700BFE4BC000038B5084BB9
:100F100090F8552053F832300124054683F80041FB
:100F20000A2005F099F900232B71204638BD00BF37
:100F3000E4BC00004079704706307047006D704790
:100F400038B50446006803681B6A98472046FFF7D7
:100F5000DDFF94F856200E4B53F83230012583F80C
:100F600080500A2005F078F92046FFF7C1FF20687D
:100F7000084B20221A6003684FF416419B6998477A
:100F800040F2EE2005F068F984F8545038BD00BFF7
:100F9000E4BC000084F00F4070B5044600680368AC
:100FA0001B6A98472046FFF7B1FF94F856200E4B76
:100FB00053F83230012283F800210A2005F04CF961
:100FC0002046FFF795FF2568084B20221A602B6802
:100FD0009E69074B186801F015FE01462846B04788
:100FE000002384F8543070BDE4BC000088F00F404A
:100FF000B888FF1F10B58EB0322201A80C4607F04A
:10100000EDFF00233A2101A88DF8353007F0A8FF45
:10101000014608B9207003E02046013107F0B7FF10
:101020000EB010BD2DE9F8430025074688469146CD
:101030000D702C462E46386803689B68984748B365
:1010400038680368DB689847C0B20EB945282DD0D0
:1010500001360D28F6B203D1002308F8043009E068
:1010600009F1FF339C42F7D008F804000134E4B2E0
:101070000025E0E7386803689B68984738B138680E
:101080000368DB6898470A2005F0E6F8F2E70120DC
:10109000BDE8F88301350A20EDB205F0DDF8312D09
:1010A000C9D9201C18BF0120BDE8F8833046BDE82F
:1010B000F883FFFF70B5044625460679FFF740FF29
:1010C000002355F81A0B0E496371FFF7F2FE204614
:1010D00029463222FFF7A6FF38B1284609490222E5
:1010E00007F065FF08B9012300E000236371204683
:1010F000FFF752FF16B92046FFF708FF607970BD71
:10110000BB9C0000B89C0000437970B50446F3B165
:1011100090F854600EB9FFF713FF25460C4955F8B7
:101120001A0BFFF7C6FE322229462046FFF77AFF48
:1011300020462946FFF75EFFA01D2946142207F02E
:101140004DFF26B92046BDE87040FFF725BF70BDB2
:10115000BE9C0000437970B50446EBB190F8546032
:101160000EB9FFF7EDFE25460C4955F81A0BFFF7AF
:10117000A0FE322229462046FFF754FF204629468A
:10118000FFF738FF284607F0A0FD206526B9204666
:10119000BDE87040FFF700BF70BD00BFC79C0000F6
:1011A00070B52B4D01600446286801F034FD03281A
:1011B00004D1212384F85530172306E00438012890
:1011C00037D8032384F85530182384F8563094F820
:1011D0005600012104F022FF94F856201D4B53F8CD
:1011E0003230012183F8001194F8550004F016FF05
:1011F0002046FFF77DFE2046FFF75CFF637933B39F
:101200002046FFF79DFE2046FFF7A4FF2046FFF78C
:101210007BFF2046FFF7C0FE2046FFF769FE2468EB
:10122000286823689E6901F0EDFC01462046B0471E
:101230000DE00A2003F024FC074B063403F11402EE
:1012400053F8041B44F8041B9342F9D170BD70BDE0
:10125000B888FF1FE4BC0000D09C0000F8B54379BB
:1012600004460F4643B390F854600EB9FFF768FE8A
:1012700025463A461149206807F0BAF855F81A0B86
:101280000F49FFF709FE204629463222FFF7CAFE22
:1012900060B128460B49022207F089FE30B9A01D33
:1012A0003946142207F09AFE012500E0002516B900
:1012B0002046FFF771FE2B461846F8BDE49C00005F
:1012C000B59C0000B89C0000437970B504460D46FB
:1012D0002BB390F854600EB9FFF732FE2A4625462C
:1012E0001049206807F084F855F81A0B0E49FFF7EB
:1012F000D3FD204629463222FFF794FE48B1284606
:101300000A49022207F053FED0F1010538BF00253B
:1013100000E0054616B92046FFF73EFE2B4618466C
:1013200070BD00BFA69C0000B59C0000B89C0000EA
:10133000F8B5437904460F4623B390F854600EB9CC
:10134000FFF7FEFD25463A460F49206807F050F8A2
:1013500055F81A0B0D49FFF79FFD2046294632220A
:10136000FFF760FE40B128460949022207F01FFE40
:1013700010B92765012500E0002516B92046FFF7C2
:101380000BFE2B461846F8BDEF9C0000B59C0000F4
:10139000B89C0000F8B5437904460F4600F11A05E1
:1013A0000BB9837615E090F854600EB9FFF7C8FDCD
:1013B00039462068FFF770FD07492068FFF76CFD8C
:1013C000204629463222FFF72DFE16B92046FFF7A8
:1013D000E3FD2846F8BD00BFB59C000000230121B5
:1013E00010B50A460446C3600361094B4FF4BF7051
:1013F00003F07AFB042120600122064B4FF4BF70FA
:1014000003F072FB42236060A360204610BD00BF62
:10141000FC9C00000D9D00000A23034AB1FBF3F180
:10142000B2FBF1F38360704730D4050010B5044679
:10143000006807F09BFC606807F098FC204610BD30
:1014400003690268D154084A03691168426842F886
:1014500023105A1CB2F5BF7FA5BF6FF4BE729B1854
:1014600002610361704700BFD489FF1FC26803692E
:101470009A42CABFC2F5BF72C2EB0300D0187047D0
:1014800038B50D460446FFF7F1FF854204DB062020
:1014900003F0F6FA002038BDE16823682944B1F56D
:1014A000BF7FA8BFA1F5BF71585C38BDC368006994
:1014B0005A1E48BF03F27D12131A58425841704712
:1014C0000023C3600361704738B50D460446FFF73B
:1014D000CDFF854204DD0820BDE8384003F0D0BAD6
:1014E000E1682944B1F5BF7FA8BFA1F5BF71E160F4
:1014F00038BDFFFF38B50B4B1D6883680446ED1AF5
:101500002046FFF7B3FF00280ADDE268636853F85E
:101510002230AB4204D820460121FFF7D5FFEFE788
:1015200038BD00BFD489FF1F014B0360704700BF67
:10153000609D0000014B0360704700BF609D00008C
:1015400010B5034B0360044606F019FF204610BD9A
:10155000609D000010B5034B0360044606F00FFFCA
:10156000204610BD609D000030B585B004AC04E994
:101570000E00089C34B94068194905B0BDE83040F8
:1015800006F036BF9DF80430022B07D0032B1DD187
:101590001449627C406806F02BFF1BE0E268637C24
:1015A000012A04D1A26840680F4912780BE0022A90
:1015B00007D1A16840680A784D780B4902EB0522F3
:1015C00001E04068094906F013FF03E008480949B3
:1015D00006F00EFF204605B0BDE8304007F0C6BB60
:1015E000909D000096A400009B9D0000A69D000019
:1015F000D091FF1FBE9D0000F8B5124F124B036043
:101600000025FA26044680F87A5080F88E50416012
:10161000426680F8485080F86050C6662A463B46CD
:101620003046012103F060FAC4F880602067012190
:1016300030462A463B4603F057FAC4F88400204659
:10164000F8BD00BFEA9D0000809D00004068014990
:1016500006F0CEBEFA9D00002DE9F041244BDFF8E4
:1016600094801B888AB005A9ADF81430D8F80030F2
:101670001A6800910221002400F168070191D569E0
:101680008DF81D40184639460322FE23A8476D46B3
:1016900007AE45F8044B96E8070085E807002346A7
:1016A000D8F800003946224603F0A8F9D8F800001F
:1016B0008DF819401E238DF818308DF81A4006AAAF
:1016C0000368009203220192D3F81CC03946FE231E
:1016D000E047009496E8070085E807002346D8F81D
:1016E00000003946224603F089F90AB0BDE8F081CE
:1016F000709D0000C088FF1F4068014906F078BE59
:10170000899E00000A4B10B5044618680023C218D1
:10171000013300210A2B82F88A10F8D1054B186892
:1017200002F00EFE60680449FFF7C3FB10BD00BF66
:10173000B888FF1FC088FF1F009F00002DE9F341FC
:10174000694D6A490446406806F052FE286866689A
:1017500001F06DFA66490246304606F049FE6549D9
:10176000606806F045FE2868666801F054FA624930
:101770000246304606F03CFE2868666801F051FAE1
:101780005E490246304606F033FE2868D4F80480ED
:1017900001F056FA0746286801F058FA064628680C
:1017A00001F05AFA3346564900903A46404606F050
:1017B0001FFE2868666801F05BFA5249024630460F
:1017C00006F016FE286801F04DFA10B160684E4927
:1017D00001E060684D4906F00BFE4D496068FFF777
:1017E0005BFB2868666801F049FA4A4902463046C0
:1017F00006F0FEFD2868676801F0D2F90646286801
:1018000001F0CBF9324603464349384606F0F0FD75
:101810002868676801F0CAF90646286801F0D9F916
:10182000324603463D49384606F0E2FD28686668C0
:1018300001F0D2F93A490246304606F0D9FD28684F
:10184000666801F0CCF9374B374A3849002818BF91
:101850001A46304606F0CCFD35496068224EFFF747
:101860001BFB2868D4F8048001F0C6F907462868F5
:10187000304D01F0BEF9304903463A46404606F085
:10188000B7FD2868FFF756FB38B32C496068FFF7AF
:1018900010FB3068D4F8048001F0B7F907463068CF
:1018A00001F0B0F93A4603462549404606F0A0FD4E
:1018B00028686668FFF740FB22490246304606F07A
:1018C00097FD28686468FFF739FB1F4902462046E8
:1018D00002B0BDE8F04106F08BBD60681B49FFF720
:1018E000E8FA02B0BDE8F081B888FF1F449F00000D
:1018F000619F0000979F0000B49F0000C59F0000FB
:10190000E09F0000FC9F00001FA0000056A0000008
:101910008DA00000B5A000005BA10000CEA00000DB
:10192000F4A000003D9F0000419F00000DA10000B9
:1019300026A10000B088FF1F4DA100007BA1000080
:10194000AAA10000D3A10000EFA100000DA2000099
:101950002DE9F0416F4D2B680446D3F8B40003F035
:1019600083F86D490746606806F042FD2B68D4F89D
:101970000480986803F06EF80A2690FBF6F2674937
:10198000404606F035FD97FBF6F206FB12736449FC
:101990006068644F06F02CFD2B686349D3F8AC20D7
:1019A000606892FBF6F206F023FD2B685F49D3F8DE
:1019B000A42060685E4E06F01BFD2B685D49D3F8DD
:1019C000A020606806F014FD2B685B491A7B6068F4
:1019D000002A0CBF3A46324606F00AFD2B685749EA
:1019E0001A69606806F004FD2B6855495A691B693D
:1019F0006068D21A06F0FCFC2B6852491A7E6068B7
:101A0000002A0CBF3A46324606F0F2FC2B684E49DB
:101A1000DA69606806F0ECFC2B684C491A6A606869
:101A200006F0E6FC4A49606806F0E2FC494B4A4988
:101A30001A78606806F0DCFC484B49491A786068FF
:101A400006F0D6FC474B48491A78606806F0D0FC8F
:101A50004649606806F0CCFC2868666801F00EF91B
:101A600043490246304606F0C3FC00262B68334447
:101A700093F88A202AB160683E4993F8943006F0C2
:101A8000B7FC01360A2EF1D160683B4906F0B0FC84
:101A9000012628686768821992F87F1006F10B0208
:101AA00050F8228049B101F0E3F80146404602F0C7
:101AB000E0FF32490346384608E001F0D9F8014614
:101AC000404602F0D6FF2E490346384632460136DC
:101AD00006F08EFC0B2EDCD12A4D2868FFF72AFA7F
:101AE00090B129496068FFF7E4F928686468FFF756
:101AF000FDF9264B264A2749002818BF1A462046DA
:101B0000BDE8F04106F074BC60682349FFF7D1F9E5
:101B1000BDE8F081B888FF1F42A2000051A200007A
:101B200070A20000419F000091A20000BBA2000033
:101B30003D9F0000DBA20000F9A200001CA30000F2
:101B400043A300006DA300008FA30000B0A300001A
:101B5000D1A30000EC91FF1FEDA30000D488FF1F6C
:101B600013A40000ED91FF1F39A400005EA4000043
:101B700083A4000093A400009CA40000ABA4000078
:101B8000DBA40000B088FF1FFAA400003BA2000005
:101B90003EA2000029A500000DA2000038B5184B98
:101BA00045680446186801F042F81649024628467E
:101BB00006F01EFC6068144906F01AFC60681349C0
:101BC00006F016FC6068124906F012FC60681149C4
:101BD00006F00EFC6068104906F00AFC60680F49C8
:101BE00006F006FC60680E4906F002FC60680D49CC
:101BF00006F0FEFB60680C49BDE8384006F0F8BB13
:101C0000B888FF1F45A500006FA5000040A6000092
:101C100053A6000060A6000079A600009BA6000065
:101C2000C7A60000E5A6000004A7000070B5234D7C
:101C300046680446286800F0FAFF2149024630460B
:101C400006F0D6FB60681F4906F0D2FB60681E49AB
:101C500006F0CEFB60681D4906F0CAFB60681C49AF
:101C600006F0C6FB1B49606806F0C2FB2868666880
:101C700000F0FBFF18490246304606F0B9FB6068E9
:101C8000164906F0B5FB6068154906F0B1FB6068BF
:101C9000144906F0ADFB6068134906F0A9FB6068C3
:101CA000124906F0A5FB6068114906F0A1FB6068C7
:101CB0001049BDE8704006F09BBB00BFB888FF1F0D
:101CC00052A700007BA70000BAA70000CEA7000023
:101CD000F5A700001AA8000053A800009BA8000068
:101CE000DEA8000065A90000D0A900000EAA00002F
:101CF0004BAA00007DAA00004068014906F078BBAD
:101D0000B0AA00002DE9F04F03298BB004468946A4
:101D100002D0FFF7F1FF61E0006D06F0D6FF8246CA
:101D2000606D06F0D2FF2F4B5FFA8AFA8346514668
:101D3000186800F0ABFF10B960682B4904E0BBF5F0
:101D4000805F04DB6068294906F052FB46E0DFF85B
:101D5000A480274BD8F800001B88ADF8143005AAE2
:101D6000036800920222002504F168070192DC69F1
:101D70008DF81D5039464A465346A0476C4607AE7B
:101D800044F8045B96E8070084E807002B46D8F87F
:101D9000000039462A4602F031FE8DF819B0D8F815
:101DA00000001E234FEA2B2B8DF818308DF81AB047
:101DB00006AA03688DE804023946D3F81CC04A46D7
:101DC0005346E047009596E8070084E807002B4655
:101DD000D8F8000039462A4602F010FE0BB0BDE8E4
:101DE000F08F00BFB888FF1F01AB00004DAB0000B3
:101DF000709D0000C088FF1F2DE9F041042988B0C4
:101E0000044602D0FFF778FF66E0006D06F05DFF44
:101E10000546606D06F059FF8046A06D06F055FF3F
:101E2000FF28074653DC2E4EEDB2306829465FFA94
:101E300088F800F02BFF50B38DF81080DFF8A880F1
:101E40008DF81170D8F8000004AA00238DF8153021
:101E50000368009202220192032604F16807D3F876
:101E60001CC08DF814602B466D4639463246E0475B
:101E700045F8044B08AB13E9070085E80700334633
:101E8000D8F800003946012202F0B8FD24E030689D
:101E900000F0F4FE85421AD10A2384F86830032347
:101EA00084F86A3002236367236F84F8695083F8EB
:101EB0000080236F5F70306804F1680104F17C02D8
:101EC00001F072FC6068074994F88D2002E06068B8
:101ED0000449082206F08CFA08B0BDE8F08100BF82
:101EE000B888FF1F96A40000C088FF1F2DE9F043AB
:101EF000032989B00446884602D0FFF7FDFE60E062
:101F0000006D314E06F0E1FEC5B2606D06F0DDFEFB
:101F10002946C7B2306800F0B9FE48B3DFF8B49084
:101F20008DF81070D9F80000012602228DF811609A
:101F300004A900238DF8153003688DF814208DE86E
:101F4000060004F16807D3F81CC02B466D463946DD
:101F5000E04745F8044B08AB13E9070085E80700A4
:101F60004346D9F800003946324602F047FD28E0E2
:101F7000306800F083FE85421ED10A2384F8683061
:101F8000022384F86A306367236F84F869501F70F6
:101F9000236F01225A70306804F1680104F17C0259
:101FA00001F064F9D4F8843060681A78074994F82D
:101FB0008D3006F01DFA04E060680549082206F03D
:101FC00017FA09B0BDE8F083B888FF1F9B9D000099
:101FD00096A40000C088FF1F2DE9F041042988B0B5
:101FE000044602D0FFF788FE66E0006D344F06F02D
:101FF0006CFEC5B2606D06F068FE5FFA80F8A06DF9
:1020000006F063FE29460646386800F03FFE60B3DE
:102010008DF81080DFF8B0808DF81160D8F80000DE
:1020200036128DF8126004AA032600238DF81530AD
:1020300003688DF814608DE8440004F16807D3F854
:102040001CC02B466D4639463246E04745F8044BE6
:1020500008AB13E9070085E807003346D8F800000D
:102060003946012202F0CAFC26E0386800F006FE7C
:1020700085421CD10A2384F86830032384F86A302F
:102080006367236F84F8695083F80080236F5E7064
:10209000236F36129E70386804F1680104F17C02E7
:1020A00001F082FB6068074994F88D2002E06068C7
:1020B0000449082206F09CF908B0BDE8F08100BF91
:1020C000B888FF1F96A40000C088FF1F2DE9F041CB
:1020D000032988B004460E4602D0FFF70DFE63E0E8
:1020E000006D334F06F0F1FDC5B2606D06F0EDFDF9
:1020F00029465FFA80F8386800F0C8FD40B38DF8D3
:102100001080DFF8B8800222D8F800008DF8112086
:1021100004A900238DF8153003688DF814208DE88C
:10212000060004F16807D3F81CC02B466D463946FB
:10213000E04745F8044B08AB13E9070085E80700C2
:102140003346D8F800003946012202F057FC2BE054
:10215000386800F093FD854221D1226F84F86950E0
:102160000A2384F86830022384F86A30666782F8AC
:102170000080226F5370386804F1680104F17C021A
:1021800001F074F8D4F8843060681A785B780949F3
:1021900002EB032294F88D3006F02AF904E060681F
:1021A0000549082206F024F908B0BDE8F08100BF17
:1021B000B888FF1F9B9D000096A40000C088FF1FE9
:1021C000022938B5044604D02046BDE83840FFF760
:1021D00093BD056D0E49284606F0CFFE40B90D4B64
:1021E000186801F019F860680B49FEF762FE38BD07
:1021F00028460A4906F0C1FE0028E5D1054C2068B2
:1022000000F0E4FF2068BDE8384001F013B800BFDB
:10221000B5AB0000B888FF1FB9AB0000BEAB000033
:10222000022910B5044603D0BDE81040FFF764BD95
:10223000006D06F04AFD094BC1B2186801F002F8C2
:1022400030B96068226D0649BDE8104006F0D0B88C
:1022500060680449FEF72DFE10BD00BFB888FF1F5F
:10226000C2AB000008AC0000032970B504461AD1C7
:10227000056D6B49284606F080FEC8B9656D694951
:10228000284606F07AFE18B9674B0121186807E066
:102290006649284606F071FE014620B9624B18686F
:1022A00000F0A0FC71E02046BDE87040FFF724BDBF
:1022B00028465F4906F061FEA8B9656D5949284670
:1022C00006F05BFE18B9584B0121186808E0574921
:1022D000284606F052FE01460028E4D1524B186809
:1022E00000F0F2FC51E02846524906F046FE48B99B
:1022F0004D4B606D1D6806F0E8FCC1B2284600F049
:102300007EFC42E028464C4906F037FE002841D1C9
:10231000606D06F0DEFCCF28054602DD60684749A7
:1023200035E0474B013093FBF0F006F069FA454980
:1023300006F06EFB0021064606F068FC28B1304628
:102340004FF07C5106F0A8F904E030464FF07C5184
:1023500006F0A0F906F06EFC3B4A03464FF4165116
:1023600010685943FEF7B0FF10B16068374901E0CB
:102370006068374906F03CF82B4BE9B2186800F06A
:1023800047FC60683349FEF794FD60683249FEF708
:1023900090FD70BD2846314906F0EFFD70B92A4B1B
:1023A000616D1868FEF75AFF10B160682C4901E0B2
:1023B00060682C49BDE8704006F01AB828462A49E2
:1023C00006F0DBFDC0B9606D06F07FFC42F20F73D2
:1023D0009842014602DD60682449EBE71A4D2868FF
:1023E000FEF7A6FF0028E3D028686468FEF7A6FD84
:1023F0001F49024620460FE028461E4906F0BDFD53
:1024000000287FF450AF104B616D18686568FEF7C7
:10241000C1FF194902462846BDE8704005F0E8BFF3
:102420000EAC00001AAC0000B888FF1F1EAC000004
:1024300021AC000031AC000039AC000040AC000021
:1024400080841E0000001646B088FF1F8CAC000080
:10245000ABAC0000CAAC0000B9AB0000EEAC0000B1
:10246000F5AC0000FDAC000003AD00000AAD0000BB
:1024700058AD00008FAD000099AD0000022970B585
:1024800004460D4608D1006D3C4906F076FD002853
:1024900049D102F04FFC6BE0032944D1056D384966
:1024A000284606F06AFD48B9364B606D1D6806F097
:1024B0000CFC0146284600F0B1FB59E028463249A1
:1024C00006F05BFD48B92F4B606D1D6806F0FDFB03
:1024D0000146284600F0A8FB4AE028462B4906F0B2
:1024E0004CFD48B9274B606D1D6806F0EEFB0146B8
:1024F000284600F0C0FB3BE02846254906F03DFD9C
:10250000B0B9656D2349284606F037FD08B9282083
:1025100005E02846204906F030FD48B91E2001217B
:1025200002F0EEFB24E0206D1C4906F026FD20B1F0
:102530002046BDE87040FFF7DFBB052DF8D1114DF7
:10254000606D2E6806F0C1FBC1B2304600F07BFB27
:10255000A06D2E6806F0B9FBC1B2304600F079FBE1
:10256000E06D2D6806F0B1FBC1B2284600F077FBA4
:1025700060680B49FEF79DFC70BD00BFA4AD000074
:10258000ABAD0000B888FF1FB6AD0000C4AD0000C1
:10259000D4AD0000DFAD0000E4AD0000EAAD000006
:1025A000B9AB0000F8B501230B7090F848303F2B11
:1025B00084BF03F1FF3380F8483090F8482002448C
:1025C0000023137204460E46012294F84800D9B243
:1025D00088420CD92144097A202905D12AB93278B8
:1025E00001323270012200E000220133EDE733783E
:1025F000052BA8BF0523337004F10805002384F8D8
:10260000603094F860703378BB421CD92846202192
:1026100094F8482006F0B2FB30B904EB8703013789
:10262000DD6484F86070ECE7A84201D10135E8E789
:1026300004EB87070023FD64054605F8013B94F889
:1026400060300133DBE7E46C4349204606F095FC3B
:10265000002860D02046414906F08FFC00285CD05D
:1026600020463F4906F089FC002858D020463D49C5
:1026700006F083FC002854D020463B4906F07DFC40
:10268000002850D02046394906F077FC00284CD06D
:102690002046374906F071FC002848D020463549CD
:1026A00006F06BFC002844D02046334906F065FC58
:1026B000002840D02046314906F05FFC00283CD07D
:1026C00020462F4906F059FC002838D020462D49D5
:1026D00006F053FC002834D020462B4906F04DFC70
:1026E000002830D02046294906F047FC00282CD08D
:1026F0002046274906F041FC48B32046254906F00C
:102700003CFC30B32046244906F037FC002814BFB7
:1027100001201120F8BD0220F8BD0320F8BD0420DF
:10272000F8BD0520F8BD0620F8BD0720F8BD08203B
:10273000F8BD0920F8BD0A20F8BD0B20F8BD0C201B
:10274000F8BD0D20F8BD1220F8BD0E20F8BD0F20F9
:10275000F8BD1020F8BD00BFEDAD0000F2AD0000E7
:10276000F6AD0000FDAD000003AE000015AE0000A8
:102770000BAE000011AE00001AAE000021AE00004A
:1027800011AF0000BDAD000029AE000034AE000066
:1027900038AE00003CAE000040AE000013B5044669
:1027A000606803689B689847002800F08B80606829
:1027B0000368DB689847C0B20D28F1D00A2894F866
:1027C000483001D1012B01D83F2B75D120460DF1A6
:1027D0000701FFF7E7FE122867D8DFE800F0730A69
:1027E0000E12161A1E22262A30363C424E545A60C9
:1027F00048002046FFF780FA5AE02046FFF716FA15
:1028000056E02046FFF7CAF952E02046FFF7A0F84D
:102810004EE02046FEF792FF4AE02046FEF772FFA8
:1028200046E02046FEF718FF42E02046FEF764FF30
:102830003EE020469DF80710FEF708FF38E02046EE
:102840009DF80710FFF75EFA32E020469DF807106A
:10285000FFF7B6FC2CE020469DF80710FFF70EFEB0
:1028600026E020469DF80710FFF7FEFC20E02046FA
:102870009DF80710FFF7D4FC1AE020469DF80710DA
:10288000FFF7BAFA14E020469DF80710FFF7A4FB03
:102890000EE020469DF80710FFF728FB08E02046D1
:1028A0009DF80710FFF712FC02E00D2002F0E8F897
:1028B000002384F8483005E05A1C234484F848205B
:1028C00018726DE702B010BD10B5044600F026F88E
:1028D000204610BDF0B589B06B4600248DF8154038
:1028E00043F8044B08AF06460D4617E9070083E896
:1028F0000700304629462246234600F080F809B0FA
:10290000F0BD08B500F0BDF8043008BD00F0F4B823
:1029100000F0FEB800F0F3B800F0FCB8F8B50446DB
:102920000D4616460846002228212A4B02F0DCF804
:10293000294B2061012106FB05F0002202F0D4F8AA
:1029400000236061DAB2AA4208D22269282101FB81
:1029500003220133D06096603044F3E70C2101225A
:102960001E4B284602F0C0F80C266FF00B01034600
:1029700000F10C0216FB0511606006FB0536826053
:102980005A1820691860183E5A605660282606FBBF
:102990000506283E5E5093600122691E8A4213DAC2
:1029A0000C2112FB01F601FB023C9F1911FB0211E5
:1029B00019444CF8087CB96002EB820100EBC101BC
:1029C00001329951D2B2E8E7A360E360002323709B
:1029D0002046F8BD44AE00005DAE000081AE0000B0
:1029E00010B50446406906F0C1F9206906F0BEF949
:1029F000606806F0BBF900232370204610BD2DE966
:102A0000F8439046027899460446836812B91D46F9
:102A1000E36009E0C568AA689A4205D1192002F06E
:102A20002FF80020BDE8F8832E68E368B2689B6841
:102A3000F068E3600F46331D01F1140E57F804CB24
:102A400043F804CB7745F9D1CB68B260F0609A4285
:102A5000A8BF1A463261896802F0CEFC2968089A3C
:102A600081F825902B6881F8248043F8182B09AA57
:102A700007CA83E807002378013323700120BDE8EB
:102A8000F88310B5047814B18368186810BD152058
:102A900001F0F6FF204610BD38B503788B4204469E
:102AA0000D4604DC1720BDE8384001F0E9BF19B934
:102AB00083689B6883601BE0013B994203D1C36834
:102AC0005B68C36014E0182001F0DAFFA368013DE1
:102AD00015F0FF059B68FAD15A689968916099686A
:102AE0004A60E2689168996091685A604B609360AF
:102AF0002378013B237038BD0021FFF7CDBF10B50F
:102B0000044623781BB12046FFF7F6FFF9E710BD16
:102B100000787047C36880689A68131A5842584111
:102B2000704710B580F8CA3090F8C83080F8C910E6
:102B3000044680F8CB2090F8C50093B1C943C9B2D0
:102B4000013103F087FA94F8CB1094F8C600C9431A
:102B5000C9B2013103F07EFA94F8CA10C943C9B270
:102B60000BE0013103F076FA94F8CB1094F8C6002C
:102B7000013103F06FFA94F8CA1094F8C7000131DC
:102B8000BDE8104003F066BA90F8C900704790F8AD
:102B9000CB00704790F8CA007047D0F8D00070475B
:102BA00090F8CC0070470B2002F076B890F8D40073
:102BB000704738B50546084685F8D4100C4601F034
:102BC00047FF2146C5F8D8000C20BDE8384002F088
:102BD00063B8D0F8D800704790F8DC00704790F8E0
:102BE000DE0070470A461720012102B10A4602F0B2
:102BF00003B8D0F8E000704790F8DF0070470F206E
:102C000002F04AB8D0F8E800704790F8E400704746
:102C1000102002F041B8D0F8EC007047002002F01C
:102C200055B8D0F8F0007047022002F04FB890F885
:102C3000F900704780F8F9100A201B2102F02CB827
:102C400090F8FA007047042002F026B890F8FB00D4
:102C50007047052002F020B890F8FC00704706206D
:102C600002F01AB890F8F8007047D0F8F4007047F6
:102C7000D0F8000170471A2002F028B890F8DD0063
:102C8000704780F8DD100E2002F006B859B100231D
:102C9000C21892F88A208A4203D001330A2BF7D156
:102CA00001E00120704700207047024649B100232F
:102CB0001846D31893F88A308B4204D0431C0A2B51
:102CC000F6D14FF0FF3070470A461720002101F07F
:102CD00093BF90F8FD1010B5044671B990F8A900A3
:102CE00003F09CF9D4F8EC30032B0CBF3220032006
:102CF00003F0B2FA012384F8FD3010BDF8B50446A4
:102D00000A2001F06DFF1B2884F8F90003D020464B
:102D10001B21FFF78FFF002001F068FFC4F8EC00D3
:102D2000022001F063FFC4F8F0000D2001F058FF0D
:102D300084F8DC000C2001F053FF84F8D40001F08B
:102D400087FEC4F8D8000B2001F04AFF84F8CC00BD
:102D500001F064FE0121C4F8D000172001F02EFF1D
:102D6000003018BF012084F8DE000E2001F038FF8B
:102D700084F8DD000F2001F033FF84F8DF0001F05C
:102D80004DFEC4F8E000102001F02AFF84F8E400B2
:102D900001F044FEC4F8E800042001F021FF84F8AB
:102DA000FA00052001F01CFF84F8FB00062001F06A
:102DB00017FF002184F8FC0084F8C410172001F0EC
:102DC000FDFE003018BF012084F8F80010B140F675
:102DD000FF7301E040F2FF33C4F8F430D4F8F03070
:102DE00003F001022273C3F3400222765A0701D591
:102DF000322304E01B074CBF4A234FF0FF3300256A
:102E0000C4F8AC3084F8FD501A2001F0EFFED4F87D
:102E1000F030C4F8000113F0160F0CBF002301239B
:102E200084F8C8304FF44873C4F8B8304FF4966350
:102E3000C4F8BC30012140F2DC53C4F8C0300A2091
:102E40000A46D44B01F050FED4F8EC702060032FFA
:102E500075D10223042084F8A83084F8C50001212C
:102E600003F0DCF8052084F8C600012103F0D6F851
:102E7000062084F8C700012103F0D0F82A46772302
:102E800020463321FFF74DFE12200121607303F02D
:102E9000C5F82520A07302F06BFC192360616376EE
:102EA00020610F230B20A376012184F8AA00242699
:102EB00003F0B4F81D2084F8B060207102F058FCD3
:102EC000A06094F8B00002F053FC1A2384F8243078
:102ED0001C2384F82530152384F82630102384F829
:102EE00027301F2384F8A9302946C4F8B40084F899
:102EF000286084F8296084F82A6084F82B6084F8BC
:102F00002C6084F82D6084F89E6084F89F6009200E
:102F100003F084F82946202003F080F8294638463B
:102F20009D4D03F07BF880260C20012103F076F8FC
:102F30002E601320012103F071F82E600AE1042FA6
:102F400070D1022384F8A830384684F8C570012176
:102F500003F064F8052084F8C600012103F05EF850
:102F6000062084F8C700012103F058F8FF222B4601
:102F700020462946FFF7D5FD1E206073012103F08E
:102F80004DF81D20A07302F0F3FB192360616376F6
:102F90002061212320200121A37684F8AA0003F0D8
:102FA0003DF81F230F2084F8B030207102F0E0FBC1
:102FB000A06094F8B00002F0DBFB1C2384F82430FE
:102FC0001B2384F82530242384F82630252384F815
:102FD0002730112384F82830132384F82930142350
:102FE00084F82A30152384F82B30172384F82C30EA
:102FF000162384F82D30122384F89E301A23C4F847
:10300000B40084F89F301020012103F007F829460E
:10301000102002F0E3FF0E2084F8A900294602F0F8
:10302000FDFF97E0052F40F091800223152084F8E2
:10303000A83084F8C500012102F0F0FF384684F87A
:10304000C670012102F0EAFF062084F8C7000121C2
:1030500002F0E4FFFF222B4620462946FFF761FDE0
:1030600014206073012102F0D9FF1020A07302F038
:103070007FFB1923606163762061212320200121D9
:10308000A37684F8AA0002F0C9FF1F230F2084F85A
:10309000B030207102F06CFBA06094F8B00002F038
:1030A00067FB1C2384F824301B2384F82530242359
:1030B00084F82630252384F82730112384F828301B
:1030C000132384F82930232384F82A30222384F818
:1030D0002B30172384F82C30162384F82D3012233C
:1030E000C4F8B40084F89E300E201A2384F89F3070
:1030F00084F8A900294602F091FF0920012102F07D
:103100008DFF2946092002F069FF0B20012102F002
:1031100085FF29460B2002F061FF0C20012102F0FF
:103120007DFF29460C2002F059FF1D20012102F0ED
:1031300075FF29461D2002F051FF1E20012102F0DB
:103140006DFF1E20294602F049FF03E0FE23C4F86C
:10315000EC3039E02046FFF7BCFD207902F008FB97
:10316000237EA06043B1607E04F0FAF8E061A07EA7
:1031700004F0F6F8206201E0E3612362237B6BB187
:10318000607B012102F04AFFA07B02F0F1FA20618E
:10319000236904E003AF000088F00F4023616361FE
:1031A00004F10A062546002385F88A30A36595F8C0
:1031B000240085F880302F1B02F0DAFA0C37013535
:1031C000B54244F82700EED12046F8BD10B5D0F83E
:1031D000EC30032B04464FF0010190F8A9000AD10E
:1031E00002F01CFF94F8A9200A4B53F83230012258
:1031F00083F8802006E002F011FF94F8A900002176
:1032000002F0ECFE002384F8FD300A20BDE81040F7
:1032100003F022B8E4BC000010B50446FFF7D6FF67
:103220004FF47A7003F018F82046BDE81040FFF71D
:1032300050BDFFFF014B024A1A6070470CED00E0E1
:103240000400FA0511F0E0020ED10B4633B113F081
:10325000010F1CBF0132D2B25B08F7E7022A03D18B
:1032600080F8C41001207047002070472DE9F74F07
:103270008B68144693F800905A78636809F1FF3A16
:103280009A42B8BF13469A444FF00008DBB2E3609D
:1032900084F811800546FFF7EBFC5FFA8AFA0746CF
:1032A00009EB0803DBB2534500F270825FFA88F63F
:1032B000B82B00F26582DFE813F0B9004301BC00CF
:1032C000C200C800630263026302CE00D40063023E
:1032D00063026302630263026302DE00630263024D
:1032E0006302E40063026302630263026302630237
:1032F00063026302630263026302630263026302A6
:103300006302630263026302630263026302EA0010
:10331000F1006302630263026302630263026302F9
:103320006302630263026302630263026302630275
:103330006302FA006302000106010C011201180188
:1033400063021E012E0163023501430163023B014A
:1033500063023D01430163024601630249015101D9
:1033600063024F0163025101700154015B0162016C
:103370006901630275017801830163028E01910185
:1033800098019F01A6016302AD01B501BD01CA010B
:103390006302DA01DE01E201E601EA01EE01F20177
:1033A000F601FA01FE01020206020A020E021202F0
:1033B00016021A021E022202290263023302360298
:1033C00039023C023F024202450248024B024E02D1
:1033D00063026302630263026302630263026302C5
:1033E00063026302630263026302630263026302B5
:1033F00063026302630263026302630263026302A5
:103400006302630263026302630263026302630294
:1034100063026302630251026302530263025602B3
:103420006302590263025C0263025F02A368952291
:10343000A8E12846D4F808B0FFF7F9FB6DE128466B
:10344000D4F808B0FFF71AFC67E12846D4F808B0B2
:10345000FFF7A6FB61E12846FFF704FCA368FF2203
:1034600090E12846D4F808B0FFF7FCFB00280CBF19
:1034700003230F23F8E02846D4F808B0FFF7ACFB8D
:103480004BE12846D4F808B0FFF7ECFB45E1D5F84E
:10349000B400D4F808B001F0E7FA3EE1A868D4F827
:1034A00008B001F0D7FA0A2390FBF3F035E1284683
:1034B000D4F808B0FFF7AFFB2FE12846D4F808B0E6
:1034C000FFF7AFFB29E12846D4F808B0FFF7A9FBC6
:1034D00022E12846D4F808B0FFF7B2FB1DE12846E8
:1034E000D4F808B0FFF7B2FB17E12846D4F808B0CB
:1034F000FFF7B2FB11E1A26801922846FFF747FBF4
:1035000083462846FFF740FB2BF00F03019A03EB9D
:103510002010905537E12846D4F808B0FFF73AFB61
:103520000011FAE02846D4F808B0FFF758FBF4E0A1
:10353000984B09E02846D4F808B0FFF75DFBECE0B3
:10354000A36801221EE1944B1A7817E12846D4F8AB
:1035500008B0FFF75AFBE0E0904BF5E7A3680322C1
:1035600010E18F4BD4F808B01868FDF7E3FCD4E005
:103570008B4BD4F808B01868FDF7B8FCCDE0884B49
:10358000D4F808B01868FDF7D9FCC6E0844BD4F82D
:1035900008B01868FDF7D2FCBEE0824B1B6893F8B8
:1035A000C420EBE0A3682A7BECE02846D4F808B0FE
:1035B000FFF758FB6A692B69D31A23EAE37340E0EB
:1035C0002846D4F808B0FFF74DFB6A692B69D31A77
:1035D00023EAE37342E0A3682A7ED3E02846D4F8C6
:1035E00008B0FFF73FFBEB692BE02846D4F808B0A2
:1035F000FFF738FBEB6931E02846D4F808B0FFF755
:1036000031FB2B6A1DE02846D4F808B0FFF72AFBEF
:103610002B6A23E02846D4F808B0FFF723FBD5F83F
:10362000A4300EE02846D4F808B0FFF71BFBD5F80D
:10363000A43013E02846D4F808B0FFF713FBD5F800
:10364000A03008B1DBB20FE0C3F387030CE02846DB
:10365000D4F808B0FFF706FBD5F8A03010B1C3F3DB
:10366000072301E0C3F387230BF806308BE0D4F87F
:1036700008B0286B46E0D4F808B0286B49E0D4F8CD
:1036800008B0686B3EE0D4F808B0686B41E0D4F84D
:1036900008B0A86B36E0D4F808B0A86B39E0D4F8CD
:1036A00008B0E86B2EE0D4F808B0E86B31E0D4F84D
:1036B00008B0286C26E0D4F808B0286C29E0D4F8CB
:1036C00008B0686C1EE0D4F808B0686C21E0D4F84B
:1036D00008B0A86C16E0D4F808B0A86C19E0D4F8CB
:1036E00008B0E86C0EE0D4F808B0E86C11E0D4F84B
:1036F00008B0286D06E0D4F808B0286D09E0D4F8C9
:1037000008B0686D394601F0B4F906E0D4F808B0A5
:10371000686D394601F0ADF900120BF8060032E091
:1037200095F88A202AE095F88B2027E095F88C20E0
:1037300024E095F88D2021E095F88E201EE095F884
:103740008F201BE095F8902018E095F8912015E067
:1037500095F8922012E095F893200FE02B68F3E69D
:103760002B685A780AE02B689A7807E02B68DA7899
:1037700004E02B681A7901E02B685A79A36801E00C
:10378000A36800229A5508F1010889E503B0BDE855
:10379000F08F00BFEC91FF1FD488FF1FED91FF1F3A
:1037A000B088FF1FB888FF1F2DE9F74F8B6893F88B
:1037B00000A0CB680AEB030B0027ABF1020B054618
:1037C000894616465FFA8BFBD7605774B846FAB243
:1037D00002EB0A03DBB201325B45D2B200F2FA809F
:1037E000D9F80810822B8C5C00F0CD803ED8442B99
:1037F00000F08B8015D8052B00F0EA8009D8032B48
:1038000065D0042B40F0E08028462146FFF7CBF935
:10381000DEE0142B6DD0432B73D0102B40F0D480FE
:1038200060E05A2B00F08B8018D8572B00F09B805B
:10383000592B7BD0452B40F0C7802846FFF7A4F9D1
:10384000014628460191FFF7A2F904F00F0404EBAA
:103850000413024601992846DBB264E0802B00F095
:10386000898000F28D805B2B6BD0ADE0892B00F05E
:10387000998015D8852B00F08C8009D8832B00F017
:103880008580842B08BF85F88D4000F0A1809BE0E7
:10389000872B00F0818000F2828085F88F4097E0CE
:1038A000B22B00F0888009D8AE2B7ED0B02B7FD011
:1038B0008A2B40F0898085F8934089E0B62B7DD033
:1038C000B82B7ED0B42B7FD12B68DC7080E02846EB
:1038D0002146FFF7DBF9002876D128462146FFF77D
:1038E000D0F975E0022C6FD828462146FFF761F920
:1038F0006EE028460CB9214600E00021FFF7E4F90C
:1039000066E02846FFF788FC62E02846FFF742F9A8
:1039100004F00F01241101EB011104EB0412034622
:10392000C9B22846D2B2FFF7FCF851E02B4B186819
:1039300014B9FDF7EBFA4BE0FDF7DAFA48E0A046E0
:1039400046E008EB042142F20F73994204DC234B5A
:103950001868FDF7EDFC03E0737C43F00803737413
:103960004FF0000834E01E4B21461868FFF76AFC50
:1039700070B329E064B31B4B186800F0E1FC27E04A
:1039800085F88A4024E085F88B4021E085F88C405A
:103990001EE085F88E401BE085F8904018E085F821
:1039A000914015E085F8924012E02B681C700FE002
:1039B0002B685C700CE02B689C7009E02B681C7114
:1039C00006E02B685C7103E0737C43F008037374BA
:1039D0000137FCE603B0BDE8F08F00BFB088FF1FE1
:1039E000B888FF1FC088FF1F38B5856A084B036081
:1039F00004462DB12846FEF7F3FF284604F0BFFC2D
:103A0000201DFDF713FD034B2360204638BD00BF8A
:103A100020AF0000609D000010B50446FFF7E4FFF2
:103A2000204604F0ACFC204610BDFFFF10B500227C
:103A300041600446034B0846012101F055F8A0609F
:103A400010BD00BFEA9D00002DE9F04106461B4B6A
:103A500046F8043B04469046002530460F46FDF7E5
:103A6000BDFC3046414684F82C5084F8425084F81E
:103A7000565084F86A502577FDF7CEFC04F13000EB
:103A8000A761FA21FFF7D2FF04F14400FA21FFF702
:103A9000CDFF04F15800FA21FFF7C8FF182004F009
:103AA0006CFC0F2102220646FEF70EFF0123A662E0
:103AB00084F82C5023772046BDE8F08120AF000029
:103AC00038B50446806903689B689847E8B1251DAE
:103AD0002846FDF70FFDA06903689B68984718B159
:103AE0002846FDF7E3FC38B194F82C301BB1074BA6
:103AF0001B68636238BD38BDA0690368DB689847FE
:103B0000C1B22846FDF79CFCE5E738BDD489FF1F0C
:103B100082B030B585B00C4608A981E80C006B4630
:103B200043F8040B07C983E80700064B9DF82C20D7
:103B300018682146032300F061FF05B0BDE830405E
:103B400002B07047C088FF1F10B586B000240193F3
:103B5000059B00938DF80D408DF80C2003AB0CCB2A
:103B6000FFF7D6FF06B010BD10B50446806AFEF719
:103B7000D1FE002384F82C3010BD38B54C78CB68CA
:103B800002341C440B780A2B0D46E4B201D18B7829
:103B900002E0142B03D14B7C1C44E4B202E00E2063
:103BA00000F06EFFE96800238B4205DAAA68D25C58
:103BB0001444E4B20133F7E7E043C0B238BD8329CF
:103BC00006D003D80139022904D801E0922901D195
:103BD000012070470020704738B5044680690368AB
:103BE0000D461B68FF219847A0690368FF211B68E9
:103BF0009847A069697803681B689847A069E968D5
:103C0000036802311B68C9B29847A069697C0368E0
:103C10001B689847A069A9680368EA685B689847C9
:103C2000A069297C03681B68984738BD70B51423C8
:103C300080F844308B780022013B04460D4680F822
:103C40005520052B26D8DFE803F003081325251E91
:103C50006B7880F8453002651CE06B7880F8453061
:103C60001F4B2946186804F14402FFF7FFFA11E0E0
:103C70006B7880F845301A4B2946186804F14402E5
:103C8000FFF792FD06E0164E3068FFF79FFA3068A6
:103C9000FFF7D0FA94F84530FE2B1FD0AB7CEBB980
:103CA0000F4E3068FEF798FF022809D03068FEF703
:103CB00093FF0128AB7801D1022B01D0012B0DD14C
:103CC00004F1440529462046FFF757FF84F85400C5
:103CD00029462046BDE87040FFF77EBF70BD00BF9B
:103CE000B888FF1F2DE9F04F8B6885B01A7893F8DC
:103CF00001B0039207460D460224EB689C4246DA67
:103D0000DFF89480AB68D8F800001E5DFEF7B6FFC0
:103D100086420BF1010A05D0D8F800003146FEF7C3
:103D2000B5FF00B3AB68039A1A551A4B1868AB6815
:103D30000268234400935FFA8AF3019307F158095C
:103D4000D2F81CC0494603223346E047D8F80000A9
:103D5000FEF794FF864209D1012387F86A3038467E
:103D60004946FFF763FF5444E4B2C6E70A4B3146C5
:103D70001868FEF78BFF30B138464946022201230E
:103D8000FFF7E2FEEFE7122000F07AFEEBE705B066
:103D9000BDE8F08FC088FF1FB888FF1FF8B5044644
:103DA000A06AFEF7B5FD002804DC2046BDE8F84017
:103DB000FFF7DABEA06A174FFEF7A3FD4578064667
:103DC0003868FEF75BFF85423146204602D1FFF797
:103DD0002DFF03E003220123FFF7B6FEA06AFEF7E2
:103DE00095FD0D4B38681B686362FEF747FF8542FF
:103DF0000FD1A06AFEF78CFD002806DDA06AFEF751
:103E000080FDC37CAB42CBD0F8BD94F82130AB42EF
:103E1000CBD0F8BDB888FF1FD489FF1F38B5012368
:103E200080F82C30084B90F820501B684362044601
:103E3000806AFEF766FD4378AB4204D12046BDE8B8
:103E40003840FFF7ABBF38BDD489FF1F2DE9F043E1
:103E50008B689B7880F820308A68CB68134485B0E3
:103E600013F8023C80F8213005460C4601264FF03D
:103E7000FF08E3689E423ADA771CDFF88490A36873
:103E8000D9F80000D95DFEF701FF38B9D9F8000074
:103E9000FEF7F4FEA368DB5D834222D1A86AFEF739
:103EA0003BFD10B11A2000F0EBFDA3689A1905F153
:103EB000580992788DF80C209A5D8DF80D200F4AE4
:103EC000DB5D106803AA0168009202220192D1F81A
:103ED0001CC04946E04785F86B80A86A4946FEF752
:103EE000F9FCA368033613F80780F6B2C1E7284649
:103EF000FFF794FF05B0BDE8F08300BFC088FF1F47
:103F0000B888FF1F037F2DE9F0470446002B00F01F
:103F1000DF8090F82C302BB16E4B1A68436AD31AAD
:103F2000642B19D82046FFF7CBFD251D2846FDF749
:103F30009DFA05280EDD28460021FDF7A1FAFF288D
:103F400040F0C18028460121FDF79AFAFF2840F091
:103F5000BA8004E0BDE8F087FFF706FEE2E7022141
:103F60002846FDF78DFA002384F8310084F84230AA
:103F700028460321FDF784FA0128074607DD284675
:103F8000FDF774FAFB1C834203DBBDE8F087BDE854
:103F9000F08794F82C304BB1142384F83030284645
:103FA0000421FDF76DFA84F8410008E00A2384F843
:103FB000303028460421FDF763FA84F83200626B42
:103FC000BB1E9342A8BF134603F10508E3635FFAE3
:103FD00088F80526F3B243450BD231462846D4F87B
:103FE0003890FDF74DFAA6F1050A013609F80A00E6
:103FF000F0E741462846FDF743FA04F1300684F81D
:10400000400031462046FFF7B8FD94F84030834227
:1040100059D194F82C3083B1A06AFEF779FC0028BE
:1040200045DDA06AFEF76DFC94F83130C27C9A42FF
:104030003DD12046FFF7B2FE42E0204694F8321010
:10404000FFF7BDFD00283BD0DFF88C8094F831905D
:10405000D8F80000FEF712FE814523D0D8F8000002
:1040600094F83110FEF712FE034630B101222046CB
:1040700031461346FFF768FD22E094F83120FE2A0E
:104080001ED194F83220832A2046314602D1FFF710
:1040900029FE15E0922A02D1FFF7D8FE10E0022295
:1040A000FFF752FD20463146FFF7C0FD08E094F8C7
:1040B000212094F831309A4202D12046FFF754FD76
:1040C0002846391D01E028460121FDF7FDF92CE7BE
:1040D000BDE8F087D489FF1FB888FF1F30B585B0D1
:1040E00004AD05E90E00089D9DF804300446002D3E
:1040F00034D0012B05D1294605B0BDE83040FFF78B
:104100006BBD032B22D190F82C30A3B12946FFF7C9
:1041100063FD134BA06A1B686362FEF7F9FB00287E
:1041200009DDA06AFEF7EDFB6B78C27C9A4202D1F2
:104130002046FFF733FE6A7894F821309A420DD179
:10414000204605B0BDE83040FFF70EBD022B05D07C
:10415000132005B0BDE8304000F092BC05B030BD82
:10416000D489FF1F38B5056D074B036004462DB198
:104170002846FDF75BF9284604F001F9204600F0D7
:104180000DFC204638BD00BF58AF000010B50446F6
:10419000FFF7E8FF204604F0F2F8204610BD2DE9B5
:1041A000F04186B004688DF814209846022205ABD1
:1041B0008E4600F13C070093019201267346394672
:1041C0008DF81560E4690546A0476C460CAB44F8D1
:1041D000048B93E80700032384E807002846394648
:1041E000324600F00BFC06B0BDE8F081F0B587B0B8
:1041F00000F13C058DF8153005AB8DF814200268F0
:104200000093022301930F46D66929463B460322B9
:104210000446B0476B460C9A43F8042B0DAA07CA14
:1042200083E80700204629469DF840209DF8443049
:1042300000F0E4FB07B0F0BDF0B587B004688DF87E
:1042400014201F46022205AB8E4600F13C06009367
:10425000019273468DF815203146E4690546A04762
:104260006C460CAB44F8047B93E80700032384E816
:10427000070028463146012200F0C0FB07B0F0BD20
:10428000F0B587B006688DF815301B128DF8142034
:104290008DF81630032205AB00F13C050093019226
:1042A0000F463B462946F6690446B0476B460C9AD2
:1042B00043F8042B0DAA07CA83E8070020462946C5
:1042C0009DF840209DF8443000F098FB07B0F0BD09
:1042D000F8B5044617460E46002500F07DFB164B48
:1042E0002360666584F8265084F83A5084F84E506E
:1042F000142004F042F80646FDF770F830463946BF
:104300002665FDF789F801220C4B08210A2000F0F0
:10431000EBFBFA21A06504F11400FFF787FB04F121
:104320002800FA21FFF782FB04F13C00FA21FFF795
:104330007DFB25712046F8BD58AF000030AF00006E
:10434000F0B51A4E054630680A2489B0224600218D
:104350008A3004F03DFD306822460021943004F09C
:1043600037FD00232A6800930124019305F13C06E0
:104370008DF815308DF81630D7698DF81440284621
:10438000314622462346B8476B468DF8174043F81E
:10439000045B08AF17E9070083E8070028463146A9
:1043A0002246032300F02AFB09B0F0BDB888FF1FA6
:1043B000F0B5002189B004465022806D04F008FD5C
:1043C000164B1B6893F88A302BB304228DF8142007
:1043D00014228DF8112004AA2168009202220025DF
:1043E000019204F13C068DF815508DF81050CF69FC
:1043F00020463146B8476B468DF8165043F8044BBB
:1044000008AD15E9070083E8070020463146012280
:10441000032300F0F3FA09B0F0BD00BFB888FF1F16
:104420002DE9F0478AB005AD85E80E009DF81430FF
:10443000129A9DF816609DF81780012B044629D129
:104440006AB1092E03D92046FFF7B2FF6FE0394960
:1044500052780968731C0E4486F88A20DEB2B8F1DF
:10446000FC0FF0D8092EEED82268002308F10108CD
:10447000009301935FFA88F804F13C07D2F81CC05E
:104480002046394601224346E0478DF816608DF8F4
:1044900017803BE0042B47D1002A48D09368876DF2
:1044A00093F8009093F801A00FFA86FC09EB0A2913
:1044B00047F83C904FEACC0107EB01089B7888F85D
:1044C0000430836D194493681B7D01360033F6B2C6
:1044D00018BF0123092E4B7129D8164B1B68334492
:1044E00093F88A301BB300228DF8242014228DF813
:1044F000252009AA01680092022200F13C070192DE
:10450000D1F81CC03946E0478DF816606B4643F879
:10451000044B95E8070083E807002046394601224E
:10452000032300F06BFA02E0042000F0A9FA0AB0BD
:10453000BDE8F087B888FF1FF0B589B004AA05234D
:104540008DF81030036800920222002400F13C062E
:104550000192DF698DF8154031468DF81140032234
:10456000FE230546B8476B4608AF43F8044B17E9EE
:10457000070083E80700284631462246234600F01C
:104580003DFA09B0F0BD38B54C78CB6802341C4414
:104590000B780A2B0D46E4B201D18B7802E0142B84
:1045A00003D14B7C1C44E4B202E00B2000F068FA1B
:1045B000E96800238B4205DAAA68D25C1444E4B2AD
:1045C0000133F7E7E043C0B238BD2DE9F0474E684C
:1045D0008D68089F0C469146002132468046284649
:1045E0009A4604F0F5FB14222046002104F0F0FB6B
:1045F0009DF8242066600A23B242A8BF3246A56017
:10460000237084F801A084F80290E2601FB128466C
:10461000394600F0F1FE40462146FFF7B4FF207412
:10462000BDE8F0872DE9F8430446006DFCF71EFF56
:10463000012827DD206D0021FCF722FFFF2805D18E
:10464000206D0121FCF71CFFFF2804D0206D012103
:10465000FCF73AFF16E0206DFCF708FF052811DD96
:104660000221206DFCF70CFF03210546206DFCF7AD
:1046700007FF0128064605D9206DFCF7F7FEF31C5D
:10468000834201DB002533E0142365752375206D1B
:104690000421FCF7F5FEA36984F82500B71E9F42AC
:1046A000A8BF1F4627620537FFB20525EBB2BB4204
:1046B0000BD22946206DD4F81C80FCF7E1FEA5F151
:1046C0000509013508F80900F0E73946206DFCF7C7
:1046D000D7FE04F11405074684F824002946204635
:1046E000FFF751FF8742206DB1D1311DFCF7ECFE81
:1046F0002846BDE8F88338B50546406D0A230B709F
:1047000003680C461B68FF219847686D0368FF210A
:104710001B689847686D617803681B689847686DE7
:10472000E168036802311B68C9B29847686DA178D7
:1047300003681B689847686DA1680368E2685B6856
:104740009847686D217C03681B68984738BD8B7853
:10475000032B11D1C86801280EDD89680B78022B64
:104760000AD918440238C0B2032805D8023BDBB28C
:104770000120CB5C13707047002070472DE9FF418A
:104780000446606D03689B68984758B1606D036884
:10479000DB689847C1B2206DFCF752FE7D4B1B6869
:1047A000A360EEE72779002F40F09180E068FEF7E4
:1047B000AFF9002840F3EA80E068FEF762F9061DD1
:1047C0000546314620460DF10F02FFF7C0FF10B33A
:1047D000714F9DF80F103868FEF758FA002840F026
:1047E000C38038689DF80F80FEF748FA804500F0D6
:1047F000BB809DF80F30002B00F0B6806979FE2950
:1048000000F0B2803F683846FEF74FFA38449DF812
:104810000F3080F88A30002385F82330AB79022BE3
:1048200038D12B69012B35DD5B4B69791868FEF7B0
:104830003CFAA36DC0B2C200991853F8303023F08F
:104840000203B3F5CA7F25D10B79142B22D8E9686E
:104850000B784978082B07D85818072804DDC3F1CE
:10486000080085F8200004E0FF20092B85F82000CF
:1048700005D81944082902DDC3F1090300E0FF232C
:1048800085F82130A36D1A44537985F822305523D9
:1048900085F82330206DFCF713FE00236B7620464D
:1048A0003146FFF728FF6B79FE2B06D1012001F07E
:1048B000D3FC20463146FFF71EFF95F824302371C4
:1048C00013B9E068FEF718F9324B1B681EE0012FA0
:1048D00046D1E068DFF8BC80FEF7D3F805462046F5
:1048E000FFF7A0FED8F80020A368064680B995F827
:1048F0002510D31A8B4249D96B7E002B38D16F76A5
:104900002046291DFFF7F7FED8F80030A3603DE0F0
:10491000214F71783868FEF7C8F9002804DB3A683F
:10492000737C104480F8943095F8233003B395F8E5
:104930002030FF2B02D0B268FF21D15495F82130EE
:10494000FF2B07D095F82210B26800290CBF032175
:104950000F21D15420463146FFF715FE307407E091
:104960000C2000F08DF811E0E068FEF7C5F80DE0CE
:10497000286830B10368009618351E6895E80E0067
:10498000B047E068FEF7B8F80023237104B0BDE833
:10499000F08100BFD489FF1FB888FF1F38B5C568F4
:1049A000064B036004462DB12846FEF719F8284649
:1049B00003F0E5FC024B2360204638BD88AF0000C1
:1049C000609D000010B50446FFF7E8FF204603F0A5
:1049D000D6FC204610BDFFFF38B5074B03600446E8
:1049E000182003F0CAFC0F210546FA22FDF796FFB6
:1049F000E560204638BD00BF88AF0000F0B505ACCB
:104A00001646059A44F8042B05460F46E8683946D1
:104A10003246BDE8F040FDF7F2BFFFFFFB280CD0A7
:104A2000FC2803D0FA2803D1054870470548704791
:104A3000054B0130B3FBF0F070470448704700BFEE
:104A400010552200C0C62D0080841E00A02526001F
:104A5000400070478010EE38024B20EAE07053F8B7
:104A600020007047B0AF000040F26B135843000BBA
:104A7000704740F2DE735843B0FBF1F07047FFFF20
:104A800070B505462C46002C23DD012D12DD134E9A
:104A9000306878B100221346FF21FEF742F84FF448
:104AA0007A7001F0D9FB002130680A460B46FEF708
:104AB00038F808E00A4B20261E604FF47A7001F0A7
:104AC000CBFB084B1E604FF47A7001F0C5FB013C34
:104AD000D9E74FF47A6001F0BFFBD3E7B888FF1F36
:104AE00084F00F4088F00F4070B51E4601FB00F4C3
:104AF00012B104F0F3F802E0204604F02FF90C495B
:104B00000B6803B908600B4D0B680860C21A2B686C
:104B100013442B60084D2B681C442C6038B907489F
:104B20000749324603F064FC1420FFF7A9FF70BD6B
:104B3000DC88FF1FD888FF1FE088FF1FD091FF1F70
:104B4000C0BB0000054B1A6840F6B7339A420146D5
:104B500002D9034803F015BC704700BFD489FF1F7A
:104B6000D091FF1F08B5084B1A6840F6B7339A4238
:104B7000014607D9054803F004FC0448BDE8084095
:104B800003F020BC08BD00BFD489FF1FD091FF1FD8
:104B900008B5084B1A6840F6B7339A42014607D960
:104BA000054803F06AFC0448BDE8084003F00ABC6D
:104BB00008BD00BFD489FF1FD091FF1F072910B582
:104BC0000C460BD872B600F02DFF62B60123A3404D
:104BD0001840C0B240FA04F4E0B210BD002010BD8D
:104BE00008B572B600F01EFF62B608BD08B572B611
:104BF00000F02CFF62B608BD2DE9FF41234D2B6864
:104C0000642B07460C4690462E460DDD204968462B
:104C100003F09AFC6846FFF795FF684603F054FCE2
:104C20002868FFF7B5FF2DE0072921D800F022FF03
:104C30000028FBD072B6384600F0F4FE62B60123BD
:104C400003FA04F418F0010F0CBF20EA0404044333
:104C5000E4B200F00FFF0028FBD072B638462146C0
:104C600000F010FF62B633680133336001200AE0C0
:104C70000849684603F068FC6846FFF773FF68461A
:104C800003F022FC002004B0BDE8F081E488FF1F9F
:104C9000ECBB000041BC000070B50B4C2368642BDA
:104CA00005460E460EDC00F0E5FE0028FBD072B68D
:104CB0002846314600F0E6FE62B6236801332360E1
:104CC000012070BD002070BDE488FF1F70B50B4C43
:104CD0002368642B05460E460EDC00F0CBFE002850
:104CE000FBD072B62846B1B200F0E6FE62B6236889
:104CF00002332360012070BD002070BDE488FF1FD7
:104D000010B5044659B101210B20FFF7C5FF002162
:104D10000C20FFF7C1FF0D200221FFF7BDFF631E2E
:104D2000DBB2FC2B05D821460E20BDE81040FFF772
:104D3000B3BF10BD08B500210220FFF7C7FF002157
:104D40001720FFF7C3FF002101221720FFF754FFB0
:104D500001210A461720FFF74FFF41F244611A2054
:104D6000FFF7B4FF03210F20FFF796FF1020014645
:104D7000FFF792FF01211320FFF78EFF012114207E
:104D8000FFF78AFF03211520FFF786FF0321162076
:104D9000FFF782FF01200146BDE80840FFF7B0BFE2
:104DA00010B572B6094B0A4C01221A702078022104
:104DB00001F034F9074A084900231370074A1370B9
:104DC0002078022201F024F862B610BD1C89FF1F72
:104DD0000289FF1F1989FF1F514E0000EC88FF1F39
:104DE000054B1A7810B51C4612B1044803F0B4FA0A
:104DF0000023237010BD00BF0189FF1F0489FF1F1E
:104E000010B5044603F0A8FA204610BD0B4B1A78E3
:104E100010B51C460AB1FFF7E3FF094B094A1B68AE
:104E2000591E914206D830225A4307480749013A91
:104E300003F07CFA0123237010BD00BF0189FF1F1E
:104E4000E888FF1F575555050489FF1F7D4E000058
:104E500008B572B6064B187801F020F8054B02220F
:104E60001A70054B03221A70FFF7D0FF62B608BD17
:104E70000289FF1F1C89FF1F1889FF1FF8B53B4CD3
:104E80002378012B274603D1BDE8F840FFF7A8BFE0
:104E9000374D2B78013BDBB22B702E46002B64D1B3
:104EA0002278D2B2022A32D1324B1978324B53F8DF
:104EB000313093F80002314B19780729C0B218D964
:104EC000012810D12E4B2F491A7808782E49D2B2DA
:104ED000C0B2885419781422013191FBF2F002FB20
:104EE0001012D2B21A70FFF75BFF04233B7001234C
:104EF00034E01978C9B24C1CE4B21C70214B1C7808
:104F000000FA01F12143C9B219702A70F8BD237863
:104F1000032B25D1194B1A78072A06D9FFF740FF32
:104F20000423237002232B70F8BD124A1248147810
:104F3000144AE4B2117850F8340011F0010F4FF028
:104F4000010114BF80F8801080F800111178490821
:104F500011701A780132D2B21A7002233370F8BD80
:104F60002378042B04BF01232370F8BD1C89FF1F85
:104F70001889FF1F0289FF1FE4BC0000EC88FF1F97
:104F80001A89FF1F1989FF1FED88FF1F38B50C4BC9
:104F90001B7804460D4613B10320FFF771FD72B66E
:104FA000084A00231370084A1370084B1C70084B02
:104FB000B3FBF5F5074B1D60FFF7F2FE62B638BD97
:104FC0001C89FF1F1B89FF1F1A89FF1F0289FF1FF2
:104FD00020A10700E888FF1F0B4B1A7810B58AB193
:104FE0001A78012AFCD172B6084CFFF7F9FE207836
:104FF00000F054FF2078022101F010F8024B00224B
:105000001A7062B610BD00BF1C89FF1F0289FF1F06
:1050100072B6054B1878054B1B78C0B2DBB262B68E
:10502000C01A18BF012070471B89FF1F1A89FF1F74
:1050300010B5FFF7EDFF80B172B6084B08491A783A
:10504000D2B2885C19781422013191FBF2F402FB90
:105050001412D2B2C0B21A7062B610BD1B89FF1F03
:10506000ED88FF1FF8B50746104E3578EDB2012DDB
:10507000FAD172B60E4C207800F010FF0323337083
:105080000C4B1F700C4B00221A702078294600F040
:10509000C5FF2278094B53F8323083F80051084B92
:1050A00002221A70FFF7B2FE62B6F8BD1C89FF1F1C
:1050B0000289FF1F1989FF1FEC88FF1FE4BC000055
:1050C0001889FF1F04480549054A002303708023FF
:1050D000437303F0F5BD00BF0489FF1F014E0000BC
:1050E0006087FF1F084B1A6842F480721A604FF401
:1050F000A072013A7FF4FDAF1A689205FCD4202318
:10510000013B7FF4FDAF7047005004402DE9F74F9D
:105110006A4E6B4B3268517E927E5C5C9D5CFF2CCC
:10512000814601D0FF2D02D11120FFF7A9FC316883
:10513000644A4B7E644F02EBC3035868002303604C
:10514000897E624802EBC102614952681360614B7B
:10515000620013440B605F4B6A0013443B605E4B7C
:105160001A6842F020021A6001235C4A03FA05F52E
:1051700003FA04F445EA04031360594B1A6822F059
:1051800080021A60574A1060574818608846B9F183
:10519000000F7AD0142001F05FF8FFF7A3FFD8F8D2
:1051A000003052491B889BB2ADF80030BDF800308A
:1051B000BDF800204E4B92B20A601A603A684D4921
:1051C000128892B2ADF80220BDF80220BDF802208C
:1051D00092B20A6048494FF00A0A0A609946FFF7FE
:1051E00081FFD8F80030414D1B88D9F8002038687D
:1051F000404C9BB2ADF80430BDF80430BDF804104B
:105200003E4B89B219602B684FF0060B42F20F7EBD
:105210000BFB02120EFB031342F21071B3FBF1F30E
:105220002B6003889BB24FF0070CADF80630B2FB41
:10523000FCF2BDF80630BDF80600C9F8002022686F
:105240002F4B80B20BFB0202DFF8ACB01860DBF82A
:1052500000300EFB0303B2FBFCF2B3FBF1F10520BF
:105260000AF1FF3A2260CBF8001000F0F5FF1AF0C7
:10527000FF0AB4D11E4A336811682A688A1ADA61B3
:105280002168DBF800208A1A1A62154B15491A6842
:1052900022F080021A600A6842F420620A601A68EA
:1052A00042F0D2021A60174B80221A70A3F24B33DD
:1052B0004FF400221A6003B0BDE8F08FB888FF1FDA
:1052C00098BC0000E4BC00003C89FF1F0000030301
:1052D0003889FF1F005104403880044008500440C2
:1052E000005004400450044080004D004089FF1FDE
:1052F0003489FF1F2C89FF1F2089FF1F3089FF1F62
:105300002889FF1F53E400E02C4BF7B51A6812F40C
:10531000805F1A680AD042F480521A60284B1A68DB
:10532000002001321A60FFF7F1FE45E042F400422E
:105330001A60244B1B681B889BB2ADF80430BDF883
:105340000430BDF80420204B92B21A601F4B1C6839
:105350004FF0060C07270CFB0424B4FBF7F41C6089
:105360001B4B196842F20F7606FB012242F21075C0
:10537000B2FBF5F21A60174B17491B681B889BB2EA
:10538000ADF80630BDF80630BDF806309BB20B60B4
:10539000124908680CFB0030B0FBF7F008601049B8
:1053A0000F6806FB0733B3FBF5F30B600D49096883
:1053B000A21AC31ACA610B6203B0F0BD00500440C8
:1053C0002489FF1F3889FF1F3089FF1F3489FF1F81
:1053D0004089FF1F3C89FF1F2889FF1F2C89FF1F61
:1053E0002089FF1FB888FF1F024B4FF400221A606C
:1053F000704700BF88E100E0844641EA000313F0F3
:1054000003036DD1403A41D351F8043B40F8043BCB
:1054100051F8043B40F8043B51F8043B40F8043B8E
:1054200051F8043B40F8043B51F8043B40F8043B7E
:1054300051F8043B40F8043B51F8043B40F8043B6E
:1054400051F8043B40F8043B51F8043B40F8043B5E
:1054500051F8043B40F8043B51F8043B40F8043B4E
:1054600051F8043B40F8043B51F8043B40F8043B3E
:1054700051F8043B40F8043B51F8043B40F8043B2E
:1054800051F8043B40F8043B403ABDD2303211D3CE
:1054900051F8043B40F8043B51F8043B40F8043B0E
:1054A00051F8043B40F8043B51F8043B40F8043BFE
:1054B000103AEDD20C3205D351F8043B40F8043BCE
:1054C000043AF9D2043208D0D2071CBF11F8013BCC
:1054D00000F8013B01D30B8803806046704700BF92
:1054E000082A13D38B078DD010F003038AD0C3F1A1
:1054F0000403D21ADB071CBF11F8013B00F8013B83
:1055000080D331F8023B20F8023B7BE7043AD9D341
:10551000013A11F8013B00F8013BF9D20B78037016
:105520004B7843708B78837060467047F0B5304B92
:105530001B681B06FBD42F4B1B6813F08002F6D1AF
:1055400072B62D4B1978002950D02C4908684F6845
:105550008E68CD680C693844143130440968284499
:1055600020440844C0F34E00254940F40040086040
:10557000C86A0F6B4E6B8D6BCC6B38444031304436
:105580000968284420440844C0F34E001D4940F4F3
:105590000040086001F10811143151F8140C51F861
:1055A000107C51F80C6C51F8085C51F8044C0968F7
:1055B00038443044284420440844C0F34E00124983
:1055C00040F400400860C86A0F6B4E6B8D6BCC6B6B
:1055D0003844403130440968284420440844C0F32A
:1055E0004E000A4940F4004008601A7062B6F0BDEF
:1055F00024B0034024B00B404589FF1F38B003405E
:105600002CB0034030B003402CB00B4030B00B4006
:1056100010B5204B2048214960221A70E1225A70AF
:105620001F4B204A1C78204B082C01D1012402E09A
:105630000A2C03D139240460132005E00C2C0CBF84
:1056400035243D2404601220086014601860174B54
:1056500017491B78174A03B101230B601360164BDF
:10566000164A1978164B012901D880210BE004292C
:1056700001D8842107E0082901D8852103E01029F9
:1056800094BF86218721116019600E4B01221A7088
:1056900010BD00BF0040074008B003400CB00340FD
:1056A0006887FF1F08B00B400CB00B404889FF1FF4
:1056B00020B0034020B00B406987FF1F24B0034097
:1056C00024B00B404589FF1F0C2804D9102828BF9F
:1056D0001020102307E00A2804D8092834BF082323
:1056E0000A2300E00C23094AD9B2081A1070084AAC
:1056F0001078834208D0074B11701B7813B1064B0A
:1057000000221A60FFF784BF704700BF4489FF1F63
:105710006887FF1F4589FF1F24B0034010B5114B58
:105720001B7804460BB1FFF701FF012C0E4A01D88C
:10573000002302E0042C02D8042313600EE0082C9E
:1057400003D805231360082308E0102C03D8062390
:105750001360102302E0072313602023034A137011
:1057600010BD00BF4589FF1F24B003406987FF1F9C
:105770000D2838B50FD9172801D80E380AE0A0F146
:105780001A03052B01D8093804E0A0F12203062BE7
:1057900047D81838C0B2244B1C5C244B1B780BB183
:1057A000FFF7C4FE210614D472B6214B214D1C60B4
:1057B00001232B7062B672B61D4B1B681A0601D509
:1057C0001D4B1FE02B78002BEFD062B602F0E8FEF5
:1057D000F1E772B6194B1A4D1A6814F0400F14BF56
:1057E00022F0100242F010021A60164B04F03F0241
:1057F0001A6001232B7062B672B6124B1B681B062F
:1058000008D5114B186800232B7062B60F4B1B781C
:10581000184138BD2B78002BDCD062B602F0C0FEF8
:10582000EAE7002038BD00BFBABC00004589FF1F71
:1058300000B003404789FF1F10B003400CB00B407D
:105840004689FF1F00B00B4010B00B404489FF1F7A
:105850000D2810B50FD9172801D80E380AE0A0F18D
:105860001A03052B01D8093804E0A0F12203062B06
:1058700027D81838C0B2134B1C5C134B1B780BB1E4
:10588000FFF754FE230607D472B6104B44F04004D1
:105890001C6001220E4B12E072B60E4B1A6814F017
:1058A000400F14BF22F0100242F010021A6004F000
:1058B0003F04094B44F040041C60084B01221A705D
:1058C00062B610BDBABC00004589FF1F00B003409E
:1058D0004789FF1F0CB00B4000B00B404689FF1FEB
:1058E0000D280FD9172801D80E380AE0A0F11A03A5
:1058F000052B01D8093804E0A0F12203062B26D895
:105900001838C0B2134B1B56002B08DB124B1B6818
:1059100013F0800F114B12D072B6114A07E0114BF1
:105920001B6813F0800F104B09D072B60F4A106835
:1059300000221A7062B60E4B1B78184170471B7814
:10594000002B14BF4FF0FF306FF0010070470020B4
:10595000704700BFBABC000000B003404789FF1F7A
:1059600010B0034000B00B404689FF1F10B00B4041
:105970004489FF1F084B1A6842F480521A60074B93
:105980001A78074B0AB1802200E0C0221A70054B3A
:1059900080F30C00188070472C8004404889FF1F5A
:1059A00021C00C4000C00C40024B1B78DB07FBD52C
:1059B000704700BF010002407FB5174B6A4603F1F4
:1059C00010056E4618685968144603C40833AB4284
:1059D0002246F7D1114B1A7812F0020F1D4612D051
:1059E00080229A7133229A7203225A7272B60C4C38
:1059F00046F001062046B04762B6237813F07003E4
:105A000001D0237006E044F621632A78D20701D43E
:105A1000013BFAD104B070BDD2BC000001000240CD
:105A200000000240B0F5006F10B5044609D2064BE5
:105A30001B78DB0701D4FFF7BFFF04F1A0542078E7
:105A400010BD002010BD00BF0100024040F2FE73F7
:105A5000984210B5044609D8054B1B78DB0701D4E2
:105A6000FFF7AAFF04F1A054208810BD002010BD4C
:105A700001000240024B187800F00100704700BF9F
:105A800001000240B0F5006F38B504460D460FD254
:105A9000084B1B78DB0701D4FFF78EFF04F1A054FD
:105AA0002378AB4204D02570BDE83840FFF77CBFB7
:105AB00038BD00BF0100024038B540F2FE73984285
:105AC00004460D461ED8104B1B78DB0701D4FFF7A8
:105AD00073FF14F0010F04F1A05404D12388AB42EA
:105AE00010D025800AE02378AB4202D02570FFF762
:105AF0005BFF63782D0AAB4204D06570BDE8384087
:105B0000FFF752BF38BD00BF01000240024B1A68C8
:105B100001321A60704700BFD489FF1F08B50B4CD3
:105B20002368580301D501F025FD2368590501D5E7
:105B300000F04CFE23681A0501D501F029F923680D
:105B4000DB04ECD501F092FBE9E700BF34800440B0
:105B500008B5FFF7E3FFFFFF014B10221A807047E3
:105B6000002005407047FFFF024A13681844106088
:105B7000184670476C87FF1F002070474FF0FF30BA
:105B800070474FF0FF307047FEE7FFFFEFF31383DE
:105B90009BB9EFF3108098B9EFF3058323B10F2B76
:105BA00004D9084A985C01E04FF48070EFF3118348
:105BB0003BB1834238BF184670474FF0FF30704703
:105BC00018467047F0E300E01F4B10B51C681C60DE
:105BD000E00304D51D4B1A680AB11B689847A1035E
:105BE00004D51A4B5A680AB15B689847E20704D596
:105BF000164B1A6C0AB11B6C9847A30704D5134BBC
:105C00005A6C0AB15B6C9847200704D50F4B9A6C0D
:105C10000AB19B6C9847610704D50C4BDA6C0AB14A
:105C2000DB6C9847220304D5084B5A6E0AB15B6EB1
:105C30009847630306D5054BD3F8802012B1D3F8FB
:105C40008030984710BD00BFA0A004404C89FF1FC2
:105C50002C4B10B51C681C60200704D52A4B5A6ACF
:105C60000AB15B6A9847E10604D5274B9A6A0AB1E4
:105C70009B6A9847620604D5234BDA6A0AB1DB6A4D
:105C80009847230604D5204B1A6B0AB11B6B984723
:105C9000A00604D51C4B5A6B0AB15B6B9847E10711
:105CA00004D5194BDA6B0AB1DB6B9847A20704D510
:105CB000154B9A6D0AB19B6D9847630704D5124B3B
:105CC000DA6D0AB1DB6D9847A00504D50E4BDA6E8C
:105CD0000AB1DB6E9847E10504D50B4B1A6F0AB188
:105CE0001B6F9847620504D5074B5A6F0AB15B6F6B
:105CF0009847230504D5044B9A6F0AB19B6F9847C8
:105D000010BD00BFA0B004404C89FF1F1E4B10B552
:105D10001C681C60E00704D51C4B9A680AB19B689C
:105D20009847210604D5194B5A690AB15B6998470F
:105D3000E20604D5154B9A690AB19B699847630737
:105D400004D5124BDA690AB1DB699847200704D5FC
:105D50000E4B1A6A0AB11B6A9847A10704D50B4B70
:105D60009A6B0AB19B6B9847A20604D5074B1A6D34
:105D70000AB11B6D9847630604D5044B5A6D0AB1EE
:105D80005B6D984710BD00BFA0C004404C89FF1F49
:105D9000114B10B51C681C60E00404D50F4BDA6889
:105DA0000AB1DB689847A10404D50C4B1A690AB103
:105DB0001B699847A20604D5084B1A6E0AB11B6EE0
:105DC0009847E30606D5054BD3F8842012B1D3F8E3
:105DD0008430984710BD00BFA09004404C89FF1F3D
:105DE000094B10B51C681C60A20704D5074B9A6EBE
:105DF0000AB19B6E9847E30704D5044BDA6F0AB1EA
:105E0000DB6F984710BD00BFA0D004404C89FF1F36
:105E1000212830B531D8042A2FD8DFE802F007094D
:105E2000050B03000B2306E00A2304E0082302E02D
:105E30000C2300E00923114A114D02EBC002546803
:105E4000104AC2F89C51104DC2F8A0510F4DC2F833
:105E5000A4510F4DC2F8A8510E4DC2F8AC5172B604
:105E600022680D4D22F47022226042F0807242EAD4
:105E7000034345F82010236062B630BDE4BC000047
:105E8000915D00000082FF1FC95B0000515C0000B3
:105E90000D5D0000E15D00004C89FF1F094B03EB25
:105EA000C0035A6872B6136823F0877323F48033F3
:105EB00043F080731360044B002243F8202062B645
:105EC000704700BFE4BC00004C89FF1F044B05492C
:105ED00000221A600A60044A106010221A6070479B
:105EE00014D0034004D0034000D003402DE9F0411A
:105EF00005460E4608462E4902F074FE2D4B00283A
:105F000047F6122814BF0227012708BF984600242D
:105F100028FA04F002F070FC4FF05E5102F0C4FC6D
:105F20000146304602F072FE10B90134072CEFD161
:105F300028FA04F002F060FC314602F069FD4FF0EF
:105F40007C5102F0A7FB02F09BFE4FF6FF739842D4
:105F500028BF1846EB1E012B06D8174B1749002205
:105F60001A600A60164A1BE0A5F10903012B06D945
:105F7000A5F11403032B02D96B1F012B06D8114B7B
:105F8000114900221A600A60104A09E0202D01D050
:105F9000192D0BD10E4B0F4900221A600A600E4AD0
:105FA00004F0070444EAC70710601F60BDE8F081F1
:105FB000001BB740006CDC020090034004900340DB
:105FC00008900340008003400480034008800340A1
:105FD00000800B4004800B4008800B40212810B546
:105FE00018D80D4A52F8303093F880423CB1012263
:105FF00011B183F8802010BD83F8002110BD02EBA1
:10600000C00043681A6811B142F0030201E022F0B7
:1060100002021A6010BD00BFE4BC0000212816D89F
:106020000B4A02EBC00301295B6852F8302004D10F
:1060300082F880124FF4A27208E0002082F88002F9
:1060400011B94FF4807201E040F203121A607047F8
:10605000E4BC0000282838B5604A04460B4611D13C
:1060600012780B2A04D8C2F10C0201FA02F304E000
:106070000C2A1CBF0C3A41FA02F31846BDE838401E
:10608000FFF778BC11780125002B05FA01F2D8BF83
:10609000002102DD934205D32946FFF79FFF2046EA
:1060A000294697E00338C2B2012A01D84C4A06E0DB
:1060B000202C01D0192C01D14A4A00E04A4A12682A
:1060C00002FB0332CA401D287BD8DFE800F0575F8F
:1060D0004E337A7A212A7A7A7A7A7A7A7A7A7A3C7A
:1060E000450F187A707A7A7A7A7A7A673F4B1A6013
:1060F00003F5973340F2444203F5FA735FE03C4BFB
:106100001A6003F5973340F2444203F5F87356E002
:10611000384B1A6003F5973340F2444203F5F673A7
:106120004DE0354B1A6003F5973340F2444203F5D6
:10613000F47344E0314B1A6003F59F3340F244425C
:1061400003F5F0733BE02E4B1A6003F59F3340F2EA
:10615000444203F5EE7332E02A4B1A6003F59F3395
:1061600040F2444203F5EC7329E0274B1A6003F533
:106170009F3340F2444203F5EA7320E0234B1A6058
:1061800003F580334FF45172203318E0204B1A602E
:1061900003F580334FF451721C3310E01D4B1A602D
:1061A000A3F5DB234FF45172A3F5F96307E01A4B13
:1061B0001A60A3F5DB234FF45172A3F2CC731A607B
:1061C00038BD7F2B2046D4BF00210121FFF706FFF9
:1061D00020460121BDE83840FFF720BF7087FF1F30
:1061E0000890034008800B40088003401080034063
:1061F0001880034020800340288003403080034003
:1062000038800340408003404880034010900340A2
:106210001890034010800B4018800B4072B60B4B57
:106220000B491A680B4B1B68096862B6490102D515
:10623000322A88BF0133C2F5BB326021FF32B2FB84
:10624000F1F24FF47A7000FB0320704718E000E091
:1062500004ED00E0D489FF1F38B50446FFF7DEFFE8
:10626000054624B938BD013C0AD005F57A75FFF71B
:10627000D5FF401BB0F57A7FF5D202F091F9F6E731
:1062800038BDFFFF1F4B4FF4000210B51A604FF0EE
:1062900080721A604FF000721A604FF080621A60CC
:1062A0004FF000621A60184B184A194C00204BF648
:1062B000FF71186059602823136093601361936124
:1062C00013629362136393630922226004F580547E
:1062D000043420606160A360236144F8042C04F559
:1062E000FE2420600B4801600B490B608B600B4B58
:1062F0001A60FFF78DF9FA20FFF7AEFFBDE81040F6
:1063000001F036BC08E100E0048003400C8003404B
:106310000080034008800B400C800B4000800B4045
:106320001D4B1A6842F480621A601C4A00231380D5
:106330001B4A13801B4A13701B4A13701B4A1370AD
:106340001B4B40F213321A604FF451725A60194BD2
:10635000C0F344321A70C0F347125A70022104226B
:1063600000F01F0098729A70D9745A7588221A74B6
:106370003C22DA709A7842F0A0029A709A7902F080
:10638000DF029A710C4B40226FF44A711A700B4471
:106390004FF400521A60704734800440608BFF1F36
:1063A000DE89FF1F688BFF1F628BFF1FDC89FF1FC9
:1063B00040A0044000A006402DE400E0134A93787A
:1063C00000F0030103F0EC030B43410748BF43F027
:1063D0001003937000F00F03042B0C4903D18B7949
:1063E00043F040038B715379C20603F0EF03074A71
:1063F00048BF43F0100353719379810603F0EF0314
:1064000048BF43F010039371704700BF00A00640DF
:1064100008B5114B1B685B0500D408BD0F4B1A78FB
:1064200002F0FF0312B102F0BBF8F7E70C4A4FF499
:10643000005111600B4A0C49D37040F203120A60FC
:106440004A600A4A13800A4A13800A4B1B680BB140
:1064500001221A7008BD00BF34800440DC89FF1F90
:1064600084E100E000A0064040A00440608BFF1FD4
:10647000DE89FF1FD889FF1F38B50446094B1B78FA
:1064800003F0FF05002BF9D120460121FFF7C6FDDF
:1064900020462946FFF7A2FD034B53F83420034B57
:1064A0001A6038BDDC89FF1FE4BC0000648BFF1F4D
:1064B0000D4A38B5146814F480624FF0000410D00F
:1064C00021280A4D0AD80A4A012152F830302B609F
:1064D000FFF7A4FD2B681C70012038BD2C602046FE
:1064E00038BD104638BD00BF34800440D889FF1F36
:1064F000E4BC00000E4B1B6813F4806316D0122816
:106500000C4B03D140F202310B4A04E0142809D1AC
:106510000A4A40F2023111605A7B42F001025A737A
:10652000012070475A7B02F0FE025A730020704728
:106530003480044000A006400CA0044014C0044075
:10654000F8B51F4B1B685A05064638D51D4B1B680E
:106550000BB101221A701C4B9A7942F020029A71F9
:106560001A4B1C780134802C1F4628BF0024184D7C
:106570002B78A34218D1FFF709FB40280FDC124A01
:1065800013791B06F3D52B7812490133802B28BFD2
:106590000023C95CDBB2C9B2D1712B70E7E7FF28D9
:1065A000E5DD01F0FDFFE2E70A4BF6B21E550A4BAE
:1065B00001221A70044BE4B2BC223C70DA70F8BDC0
:1065C00034800440648BFF1F00A00640688BFF1FCF
:1065D000628BFF1FE089FF1FDC89FF1F294B1B68AF
:1065E0005A052DE9F04707468A4649D5264B1B68D0
:1065F0000BB101221A70254B9A7942F020029A7150
:106600003D4607EB0A039D4237D2DFF89080204ECB
:1066100098F8004096F800900134802C28BF0024A0
:106620005FFA89F9A1451DD1184BBC22DA70FFF73A
:10663000ADFA40280FDC154A13791B060FD53378C5
:1066400014490133802B28BF0023C95CDBB2C9B2D7
:10665000D171337003E0FF2801DD01F0A1FF337831
:106660004B45E4D00B4B15F8012B1A550A4B012270
:10667000E4B21A7088F80040C3E7044BBC22DA7019
:10668000BDE8F08734800440648BFF1F00A0064003
:10669000628BFF1FE089FF1FDC89FF1F688BFF1FD4
:1066A00008B5034B1B7813B101F07AFFF9E708BD79
:1066B000DC89FF1F064A074B1B781078DBB2C0B29B
:1066C00083422CBF7F3000F1FF30C01A704700BFFB
:1066D000628BFF1F688BFF1F054B1888054B1B88BB
:1066E00080B29BB2984238BF00F58070C01A7047E4
:1066F000608BFF1FDE89FF1F114B12491A880B8820
:1067000092B29BB29A4210B516D00133B3F5807F96
:1067100028BF00230C489CB2C05C0C800B49096860
:10672000C0B259B19A4238BF02F58072D31A1A2BFF
:1067300004DC00230B7010BD4FF0FF3010BD00BF14
:10674000608BFF1FDE89FF1F608AFF1FD889FF1F34
:10675000094B1A88094B1B8892B29BB29A4208D007
:106760000133B3F5807F28BF0023054AD05CC0B257
:1067700070474FF0FF307047608BFF1FDE89FF1FAF
:10678000608AFF1F0C4B1B685B0514D50B4BDA7836
:1067900002F0CB02DA7040225A74DA7842F0340206
:1067A000DA70074B1A88074B92B21A80064B1B68A7
:1067B0000BB100221A7070473480044000A00640DC
:1067C000DE89FF1F608BFF1FD889FF1F30B53E4B4E
:1067D0001A7912F0300F32D072B69A7D02F0FF00B3
:1067E00022B9DA7940225A7462B628E062B6374A92
:1067F0003749138809889BB289B21446324AD57941
:106800005A1CB2F5807F28BF00228A42EDB202D026
:10681000304B9D541346421E12F0FF00EED19AB247
:1068200022802D4A126852B18B4236BFC1F5807169
:10683000C1EB03035B18272BC4BF01231370224B4A
:10684000D978C9B20A0620D51B791D061DD5234B60
:10685000234A1D781378EDB2DBB21046AB420CD060
:10686000194A0133802B14791E4C28BF0023E45CA5
:10687000E4B2D471127D072AF0D9DBB20370124B57
:106880001A79140644BF7C22DA700F4B9A7C5007A9
:1068900006D5154A10780130C0B2107004229A74DF
:1068A000490610D5084B1A7952060CD50F4A00211B
:1068B00011700F4A126802B111709A7902F0DF026A
:1068C0009A713C22DA7030BD00A00640608BFF1F39
:1068D000DE89FF1F608AFF1FD889FF1F688BFF1F9B
:1068E000628BFF1FE089FF1FEC91FF1FDC89FF1FF8
:1068F000648BFF1F1D4B1A6842F400621A601C4A29
:10690000002313801B4A13801B4A13701B4A137009
:106910001B4A13701B4B40F213321A604FF4517232
:106920005A60194BC0F344321A70C0F347125A70C0
:1069300000F01F000422022198729A70D9745A75CF
:1069400088221A743C22DA709A7842F0A0029A7077
:106950009A7902F0DF029A710C4B40221A70A3F26E
:106960002B334FF400421A60704700BF348004405C
:10697000748DFF1F728BFF1F7C8DFF1F768DFF1F95
:10698000708BFF1F0CB0044000B006402FE400E005
:10699000134A937800F0030103F0EC030B43410723
:1069A00048BF43F01003937000F00F03042B0C4911
:1069B00003D18B7943F040038B715379C20603F006
:1069C000EF03074A48BF43F01003537193798106E0
:1069D00003F0EF0348BF43F010039371704700BF0B
:1069E00000B0064008B5114B1B681B0500D408BD5C
:1069F0000F4B1A7802F0FF0312B101F0D1FDF7E757
:106A00000C4A4FF4004111600B4A0C49D37040F21C
:106A100003120A604A600A4A13800A4A13800A4B2A
:106A20001B680BB101221A7008BD00BF34800440FE
:106A3000708BFF1F84E100E000B006400CB0044002
:106A4000748DFF1F728BFF1F6C8BFF1F38B50446C0
:106A5000094B1B7803F0FF05002BF9D120460121DB
:106A6000FFF7DCFA20462946FFF7B8FA034B53F844
:106A70003420034B1A6038BD708BFF1FE4BC00004C
:106A8000788DFF1F0D4A38B5146814F400624FF07A
:106A9000000410D021280A4D0AD80A4A012152F8D0
:106AA00030302B60FFF7BAFA2B681C70012038BD1C
:106AB0002C60204638BD104638BD00BF34800440ED
:106AC0006C8BFF1FE4BC00000B4B1B6813F40063CE
:106AD00010D01728094B09D1094A40F20231116040
:106AE0005A7B42F001025A73012070475A7B02F030
:106AF000FE025A73002070473480044000B0064004
:106B000008B00440F8B51F4B1B681A05064638D577
:106B10001D4B9A7942F020029A711C4B1B680BB1F5
:106B200001221A701A4B1C780134802C1F4628BF92
:106B30000024184D2B78A34218D1FFF727F84028DE
:106B40000FDC114A13791B06F3D52B781249013358
:106B5000802B28BF0023C95CDBB2C9B2D1712B7076
:106B6000E7E7FF28E5DD01F01BFDE2E70A4BF6B29F
:106B70001E550A4B01221A70034BE4B2BC223C7032
:106B8000DA70F8BD3480044000B00640788DFF1FF5
:106B90007C8DFF1F768DFF1F748BFF1F708BFF1F77
:106BA000294B1B681A052DE9F04707468A4649D547
:106BB000264B9A7942F020029A71254B1B680BB143
:106BC00001221A703D4607EB0A039D4237D2DFF8D7
:106BD0009080204E98F8004096F800900134802C68
:106BE00028BF00245FFA89F9A1451DD1174BBC22AB
:106BF000DA70FEF7CBFF40280FDC144A13791B062E
:106C00000FD5337814490133802B28BF0023C95C8A
:106C1000DBB2C9B2D171337003E0FF2801DD01F0AE
:106C2000BFFC33784B45E4D00B4B15F8012B1A55BC
:106C30000A4B0122E4B21A7088F80040C3E7034B04
:106C4000BC22DA70BDE8F0873480044000B0064012
:106C5000788DFF1F768DFF1F748BFF1F708BFF1FBA
:106C60007C8DFF1F08B5034B1B7813B101F098FC16
:106C7000F9E708BD708BFF1F064A074B1B78107899
:106C8000DBB2C0B283422CBF7F3000F1FF30C01AAC
:106C9000704700BF768DFF1F7C8DFF1F054B188846
:106CA000054B1B8880B29BB2984238BF00F5C0707C
:106CB000C01A7047748DFF1F728BFF1F114B124952
:106CC0001A880B8892B29BB29A4210B516D0013343
:106CD000B3F5C07F28BF00230C489CB2C05C0C8079
:106CE0000B490968C0B259B19A4238BF02F5C07267
:106CF000D31A1A2B04DC00230B7010BD4FF0FF30A9
:106D000010BD00BF748DFF1F728BFF1FF48BFF1F20
:106D10006C8BFF1F094B1A88094B1B8892B29BB2E0
:106D20009A4208D00133B3F5C07F28BF0023054A3B
:106D3000D05CC0B270474FF0FF307047748DFF1FBA
:106D4000728BFF1FF48BFF1F0C4B1B681B0514D5A8
:106D50000B4BDA7802F0CB02DA7040225A74DA7800
:106D600042F03402DA70074B1A88074B92B21A804D
:106D7000064B1B680BB100221A7070473480044028
:106D800000B00640728BFF1F748DFF1F6C8BFF1FBE
:106D900030B53E4B1A7912F0300F32D072B69A7D70
:106DA00002F0FF0022B9DA7940225A7462B628E074
:106DB00062B6374A3749138809889BB289B21446AC
:106DC000324AD5795A1CB2F5C07F28BF00228A42C8
:106DD000EDB202D0304B9D541346421E12F0FF001C
:106DE000EED19AB222802D4A126852B18B4236BF40
:106DF000C1F5C071C1EB03035B18272BC4BF01238E
:106E00001370224BD978C9B20A0620D51B791D060A
:106E10001DD5234B234A1D781378EDB2DBB2104603
:106E2000AB420CD0194A0133802B14791E4C28BF79
:106E30000023E45CE4B2D471127D072AF0D9DBB2FE
:106E40000370124B1A79140644BF7C22DA700F4B80
:106E50009A7C500706D5154A10780130C0B21070E0
:106E600004229A74490610D5084B1A7952060CD59B
:106E70000F4A002111700F4A126802B111709A79FD
:106E800002F0DF029A713C22DA7030BD00B0064099
:106E9000748DFF1F728BFF1FF48BFF1F6C8BFF1F06
:106EA0007C8DFF1F768DFF1F748BFF1FD488FF1F03
:106EB000708BFF1F788DFF1F174B1A6842F48052AA
:106EC0001A60164A00231380154A1380154A13804E
:106ED000154A1380154A1370154A40F21331116098
:106EE0004FF451715160134AC0F344311170C0F333
:106EF000471100F01F0051709072937013742C238F
:106F0000D3700D4B40226FF44B711A700B444FF449
:106F100000321A60704700BF348004408890FF1F21
:106F2000868DFF1F9090FF1F8A90FF1F848DFF1F8B
:106F300008C0044000C0064031E400E0134A9378E2
:106F400000F0030103F0EC030B43410748BF43F09B
:106F50001003937000F00F03042B0C4903D18B79BD
:106F600043F040038B715379C20603F0EF03074AE5
:106F700048BF43F0100353719379810603F0EF0388
:106F800048BF43F010039371704700BF00C0064034
:106F900008B5114B1B68DB0400D408BD0F4B1A78F1
:106FA00002F0FF0312B101F0FBFAF7E70C4A4FF4CD
:106FB000003111600B4A0C49D37040F203120A6091
:106FC0004A600A4A13800A4A13800A4B1B680BB1B5
:106FD00001221A7008BD00BF34800440848DFF1F59
:106FE00084E100E000C0064008C004408890FF1F14
:106FF000868DFF1F808DFF1F38B50446094B1B7817
:1070000003F0FF05002BF9D120460121FFF706F818
:1070100020462946FEF7E2FF034B53F83420034B8A
:107020001A6038BD848DFF1FE4BC00008C90FF1FE8
:107030000D4A38B5146814F480524FF0000410D093
:1070400021280A4D0AD80A4A012152F830302B6013
:10705000FEF7E4FF2B681C70012038BD2C60204631
:1070600038BD104638BD00BF34800440808DFF1FFE
:10707000E4BC00000B4B1B6813F4805310D00E28A7
:10708000094B09D1094A40F2023111605A7B42F0A2
:1070900001025A73012070475A7B02F0FE025A73B4
:1070A000002070473480044000C0064004C0044003
:1070B000F8B51F4B1B68DA04064638D51D4B1B6814
:1070C0000BB101221A701C4B1C88A4B20134B4F518
:1070D000C07F1F4628BF0024184D2B889BB2A342B7
:1070E0001AD1FEF753FD402811DC154A13791B060F
:1070F000F2D52B8813499BB20133B3F5C07F28BF6B
:107100000023C95C9BB2C9B2D1712B80E4E7FF2890
:10711000E2DD01F045FADFE70A4BF6B21E550A4BF5
:1071200001221A70064BA4B2AC223C80DA70F8BD82
:10713000348004408C90FF1F9090FF1F8A90FF1FA7
:1071400000C00640888DFF1F848DFF1F38B50446A0
:107150004518AC4204D014F8010BFFF7A9FFF8E77B
:1071600038BDFFFF08B5034B1B7813B101F018FAC7
:10717000F9E708BD848DFF1F064A074B1B8810885E
:107180009BB280B283422CBF00F27F1000F1FF302F
:10719000C01A70478A90FF1F9090FF1F054B1888F8
:1071A000054B1B8880B29BB2984238BF00F5C07077
:1071B000C01A70478890FF1F868DFF1F114B124920
:1071C0001A880B8892B29BB29A4210B516D001333E
:1071D000B3F5C07F28BF00230C489CB2C05C0C8074
:1071E0000B490968C0B259B19A4238BF02F5C07262
:1071F000D31A1A2B04DC00230B7010BD4FF0FF30A4
:1072000010BD00BF8890FF1F868DFF1F088FFF1FD6
:10721000808DFF1F094B1A88094B1B8892B29BB2C5
:107220009A4208D00133B3F5C07F28BF0023054A36
:10723000D05CC0B270474FF0FF3070478890FF1F9E
:10724000868DFF1F088FFF1F054B1A88054B92B2D2
:107250001A80054B1B680BB100221A70704700BFE3
:10726000868DFF1F8890FF1F808DFF1F10B5314B4B
:107270001A79920623D5304AD87913882F499BB2C0
:1072800001330988B3F5C07F28BF002389B28B4240
:10729000C0B203D02A49C85499B21180294A116852
:1072A00069B1294A128892B2934236BFC2F5C072C0
:1072B000C2EB03039B18272BC4BF01230B701D4A8D
:1072C000D178C9B20C0618D51379180615D51F4BFD
:1072D0001D481C880388A4B29BB29C4202D16C2337
:1072E000D3700AE00133B3F5C07F28BF0023184CE8
:1072F000E45C9BB2E4B2D47103800E4B9A7C5207DB
:1073000006D5144A10780130C0B2107004229A7465
:107310004B060ED5074B1A7912F0400F194608D0CC
:107320000D4B00221A700D4B1B6803B11A702C23F1
:10733000CB7010BD00C006408890FF1F868DFF1FD8
:10734000088FFF1F808DFF1F8A90FF1F9090FF1FE7
:10735000888DFF1FED91FF1F848DFF1F8C90FF1FF5
:1073600021282BD8164B1B5CFF2B27D0154A02EB8C
:10737000C000002142681160134A106840F02000EC
:107380001060124A012011601149984008601148AC
:1073900041F8040C104911604FF4A07101397FF4D9
:1073A000FDAF11688905FCD42022013A7FF4FDAFBE
:1073B0000A4A1BB232F8130080B2704700207047AF
:1073C000F4BD0000E4BC00003880044000500440DC
:1073D000085004400000020380014A0000510440AC
:1073E000F0B50C4B0C4C1A7842F0020504EBC506C4
:1073F00082F00102706009481A700678002E0CBFF6
:107400008827C82786F0010647EA0141067044F83C
:107410003510F0BDFC90FF1F0080FF1F7491FF1F0F
:10742000431E032B10B510D872B6094A52F8230038
:1074300048B1416842F82310064A018832F81340E7
:10744000611A22F8131062B610BD002010BD00BFF3
:10745000EC90FF1FEE91FF1F013803280AD872B687
:10746000054B53F82030002013B101305B68FBE777
:1074700062B67047002070474091FF1F10B572B68A
:107480000123174A1A4412F8012C12071CD599003F
:10749000144A52F831402CB902EB431308305860BB
:1074A000114B09E041F0010152F8314064B902EB9F
:1074B000C103083058600D4B42F831300C4B1A783C
:1074C000013A1A7062B610BD0133052BD9D162B6EC
:1074D000074B00221A70BDE8104000F0A7BB00BFA8
:1074E00048BF00000080FF1F88004000C800400027
:1074F0006A91FF1F431E032B30B532D8194A400151
:1075000040F01000104472B6174CE25C032A09D810
:10751000DFE802F0160218050830022213E00830F6
:10752000042210E01148124A50F8234014B940F8E0
:10753000231002E052F82300416042F823100FE0CC
:10754000032200E00522E25410F0080F01F10803C5
:107550000A8843600CBF8823C82343EA02430360C0
:1075600062B630BD0080FF1FA890FF1F4091FF1F33
:107570005091FF1F2DE9F84FAB4F3C78E4B214F067
:10758000040F3D4619D0A94B1B78A3B1A84A117826
:1075900001F0FF0321B1013BDBB2137003B900BE60
:1075A000A44A117801F0FF0329B1013BDBB213704B
:1075B0000BB900F04FFC04233B7004F0080303F008
:1075C000FF02002B00F067829B4B9C4C1A78D2B2D2
:1075D00015094FEA920840F0E48104EBC8035968AA
:1075E00054F83830C3F38303013B0C2B00F2D681EF
:1075F000DFE813F095019501D401D401D401D40141
:10760000D401D401B001D401D401D4010D008C4DBA
:107610000A684B688B486B6001218B4B44F838300B
:107620002A60DFF85082017092B240F2816000233C
:107630008242C8F800302361A36117D8B2F5D06F39
:1076400080F01E81B2F5817F00F0CF8006D8802ABD
:1076500000F0BA80822A00F0BB8031E140F20233B0
:107660009A4200F0D180B2F5A06F1CE042F22100F6
:10767000824200F051810ED8B2F5086F00F09E8072
:10768000B2F5106F40F01C81684B6C4EAA781A70EE
:1076900006F180090AE042F221218A4200F00881C5
:1076A00042F221339A4200F00F8109E1336A1B064E
:1076B00003D5706A083800F0B9FA08364E45F5D19E
:1076C0000026B146DFF8B0A156F80A0028B1D0F87C
:1076D00004B000F0ABFA5846F8E74AF806005B4BF6
:1076E000DFF898A1F05056F80A0028B1D0F804B09D
:1076F00000F09CFA5846F8E7554B4AF80600F0505F
:10770000544B23F81900544B19F80320023A032A6A
:1077100008D8DFE802F002040204002200E001229F
:1077200003F8092009F10109B9F1040F06F1040673
:10773000C8D14A4B00221A7001269A46484A494B42
:107740003244334412F8012C9B0012F0080F1A70D7
:107750004FEA860925D000F04BFA38B104EB461306
:1077600008305860404B44F8393006E09AF8003051
:1077700044F8390001338AF8003000F039FA49F052
:10778000010338B104EBC302083050602E4A44F8BC
:10779000332006E044F833009AF8003001338AF8C9
:1077A000003049F00202013649F003090023052E9A
:1077B00044F8323044F83930C0D186E01B4B2B4CB2
:1077C0001B7823700B4683E0284C237063707EE0A7
:1077D000AA88042A74D8254C920023706370244B25
:1077E0009B5C9E0773D5217071E0AA8802F07F022E
:1077F000042A65DC6B88002B62D191001C4A0A4484
:10780000117821F0020159E0AA8802F07F02042ACF
:1078100056DC6B88002B53D19100154A0A4411782D
:1078200041F002014AE000BF802007407391FF1F32
:10783000FD90FF1F7591FF1F902007400080FF1FE4
:107840006091FF1F7491FF1FC80040009890FF1FB8
:107850005091FF1FEE91FF1FA890FF1F6A91FF1F1D
:1078600048BF000030C80110880040006B91FF1F26
:10787000C02007409490FF1FEC90FF1F4091FF1F16
:107880006A88A9889F4B53F8084CA3F10C00BCB13F
:1078900033F80C6C964209D133F80A6C8E4205D14C
:1078A000120A032A0CBF2378038911E00C33EAE79C
:1078B000954A1168954A1160A978954A117004E0BB
:1078C000944B0F221A7027E000231C4600E002238D
:1078D000EE88B34238BF1E46402E34BF35464025A1
:1078E00020462946FFF77CFD761B2C4403D1402D12
:1078F00012D1354603E0402E34BF354640252046A0
:107900002946FFF76DFD761B2C4401D1402D03D194
:10791000814AC8F8004016800122804B3DE0804B30
:107920001A8842F221039A4210D100237D4AC85C92
:1079300098540133072BF9D11368862B02D17A4B67
:107940000F221A7000200146FFF74AFD774B44F8DA
:10795000383023E0764E3568B5B1DFF8BC81B8F831
:107960000090B9F1400F34BF4C46402428462146D0
:10797000FFF736FDC4EB09039BB2A8F800300BB942
:10798000402C00D12B193360654B1A88B2F5A06FDB
:1079900004D100225A709A78664B1A7001225F4B0C
:1079A0006CE004EBC806013D736802F00802A3F125
:1079B0000800EDB202F0FF01002A36D000F036F9DF
:1079C0005D485E4B50F82520EAB1516840F825101B
:1079D00002F108017160595D03290BD8DFE801F05D
:1079E00002040608032104E0022102E0052100E070
:1079F0000421595516F0080F12880CBF8823C8239C
:107A000043EA024342E05A5D032A07D8DFE802F066
:107A100040400204002206E0012204E016F0080FB4
:107A20000CBF022203225A5532E054F83820120CBF
:107A300023F8082C22B3DFF834E123F8061C43F8BE
:107A4000041C5EF825303E4913B94EF8250002E0CB
:107A500051F8253058603B4B41F8250033F815109C
:107A60000A4423F8152000F0C3F810B10830706004
:107A700006E0354B44F838001A7801321A7007E0F6
:107A80002A4B324A16F0080F08BF134644F8383024
:107A900008233B7070E5E0071FD520492B482C4C8C
:107AA00002230B702B4B1A702B4B186098602B48DD
:107AB000D8601A619A615C60164B0D2018702848D6
:107AC000FF2303702B700274264A1370264B9F22EB
:107AD0001A7001230B70BDE8F88F210604D50D4BF9
:107AE0000D221A7080232B70A20705D51C4B1A7823
:107AF000D2B21A7002232B70E30644BF10232B70FE
:107B0000BDE8F88F58BF0000D489FF1F0092FF1F07
:107B10008491FF1FC02007406891FF1F94200740F9
:107B20006091FF1FF891FF1FFD90FF1FC8004000EC
:107B30009490FF1F982007404091FF1FA890FF1FBF
:107B40009890FF1FEE91FF1F6A91FF1F8800400071
:107B5000AC90FF1FFC90FF1F0080FF1F0091FF1FD4
:107B6000882007408C20074084200740EC90FF1FAE
:107B700008B500F053FD00221A4B0021D15098188F
:107B80000832882A4160F7D1174A106840F48020F3
:107B9000106002F528326832C3F307201070C3F377
:107BA00007401B0E10751376FF2302F81C3C02F8E9
:107BB000143C02F88C3C012302F8083C82F8641063
:107BC00002F8183C094B70226FF450711A700B4484
:107BD0004FF400721A6003F1C04303F5C82310226A
:107BE0001A7008BD0080FF1F3480044049E400E0A3
:107BF00072B60C4A1168B1FA81F30B2B02D962B646
:107C0000002070474FF00040D84021EA0001116089
:107C100062B6054948225343C8180022CA50426040
:107C2000704700BF7487FF1F0084FF1F0C4B482262
:107C3000C31AB3FBF2F30B2B11D80A4A127822B104
:107C4000094A12780AB1FFF719BC72B6074A4FF019
:107C5000004121FA03F311681943116062B67047BD
:107C60000084FF1F6A91FF1F7391FF1F7487FF1F1E
:107C700010B5104C23686BB120684288531C024435
:107C8000147A0288934212D3FFF7D0FF094B0022E7
:107C90001A600DE0084B1B7813B94FF0FF3010BD90
:107CA0000320FFF7BDFB20600028E5D1F5E7438006
:107CB000204610BD8091FF1F7391FF1F10B50B4C24
:107CC000236813B123686BB902E0094B1B7813B921
:107CD0004FF0FF3010BD0320FFF7A2FB206000280B
:107CE000F0D1F5E75A881344187A10BD8091FF1F30
:107CF0007391FF1F044B9888044B1B681BB11A88B3
:107D00005B88D31A18447047EE91FF1F8091FF1FC4
:107D10002DE9F8432D4E012307460C463370002C05
:107D20004FD02B4D2B68A9462BBB4AF2F928294B83
:107D30001B7803F0FF020BB9327015E00420FFF747
:107D40008BFB072808D801233370FFF751FFC9F8D0
:107D5000000080B91D4B1870B8F101081E4B01D00E
:107D60001A782AB101221A704FF0FF30BDE8F8836B
:107D700000F016FCDBE72968174A488800231370D7
:107D8000C0F14002944238BF224600F1080C104472
:107D90008C444880A41A934204D0F85C0CF8030089
:107DA0000133F8E71F444B883F2B06D940230B8053
:107DB0000420FFF79FFB00232B60084B05221A705D
:107DC000ADE734702046BDE8F88300BF7691FF1F11
:107DD0007891FF1F7391FF1F7C91FF1F7591FF1F0B
:107DE00007B502AB012103F8010D1846FFF790FF1C
:107DF00003B05DF804FBFFFF2DE9F041114B1B7848
:107E0000F3B1114E114B3468114D01271F70984684
:107E10004CB1002763882F70042023802146FFF790
:107E200069FB376009E0FFF7E3FE014620B104205B
:107E30002C70FFF75FFB00E02F70002388F8003004
:107E4000BDE8F0817391FF1F7891FF1F7691FF1FAE
:107E50007591FF1F38B50E4B1B7803F0FF05ABB9CA
:107E60000C4C216831B14B880B800420FFF742FB9A
:107E7000256038BDFFF7BCFE014620B10420BDE8F7
:107E80003840FFF737BB044B01221A7038BD00BFE2
:107E90007691FF1F7891FF1F7591FF1F08B503684A
:107EA000C9B21B68984708BD08B50368C9B21B680A
:107EB000984708BD08B50368C9B21B68984708BD54
:107EC00008B50368C9B21B68984708BD4B0803F1A1
:107ED000376000F5D830B0FBF1F0FEF721BA10B5ED
:107EE0004B0803F1376000F5D8301446B0FBF1F0D1
:107EF000FEF716FA2046BDE81040FEF75FBAFEF71F
:107F000087BA0846FEF7B8BA08B50846FEF7D0FAB1
:107F1000003018BF012008BD08B50846FEF7EAFA90
:107F2000003018BF012008BDFEF7D6BBFEF710BC1D
:107F3000FEF7E2BBFEF7B4BBFEF724BCFEF7BABB0C
:107F400008B50846FEF7FCFA012008BD08B508464A
:107F5000FEF7F6FA012008BD10B508461446114692
:107F6000FEF73CFB204610BD38B508460D4601F033
:107F700016F8044621462846FEF730FB204638BD59
:107F80007047FFFF044B00221A714FF47A711A7385
:107F9000024A99601A6070478891FF1F20BE000056
:107FA00008B50368C9B21B68984708BD08B50368DF
:107FB000C9B21B68984708BD08B50368C9B21B68F9
:107FC000984708BD08B50368C9B21B68984708BD43
:107FD0004B0803F1376000F5D830B0FBF1F0FEF745
:107FE00089BC10B54B0803F1376000F5D830144652
:107FF000B0FBF1F0FEF77EFC2046BDE81040FEF736
:10800000C7BCFEF7EFBC0846FEF720BD08B5084622
:10801000FEF738FD003018BF012008BD08B508463E
:10802000FEF752FD003018BF012008BDFEF736BE36
:10803000FEF770BEFEF742BEFEF714BEFEF784BE2A
:10804000FEF71ABE08B50846FEF75CFD012008BD24
:1080500008B50846FEF756FD012008BD10B50846D4
:1080600014461146FEF79CFD204610BD38B5084663
:108070000D4600F094FF044621462846FEF790FD89
:10808000204638BD7047FFFF044B00221A714FF4A1
:108090007A711A73024A99601A6070479891FF1FAB
:1080A00078BE000008B50368C9B21B68984708BDD0
:1080B00008B50368C9B21B68984708BD08B50368CE
:1080C000C9B21B68984708BD08B50368C9B21B68E8
:1080D000984708BD4B0803F1B76000F55840B0FB66
:1080E000F1F0FEF7E9BE10B54B0803F1B76000F5FB
:1080F00058401446B0FBF1F0FEF7DEFE2046BDE826
:108100001040FEF71BBFFEF743BF0846FEF774BFE3
:1081100008B50846FEF78CFF003018BF012008BDE7
:1081200008B50846FEF7A6FF003018BF012008BDBD
:10813000FFF734B8FFF76EB8FFF740B8FFF712B893
:10814000FFF782B8FFF718B808B50846FEF7B0FF8A
:10815000012008BD08B50846FEF7AAFF012008BDAA
:1081600010B5084614461146FEF7F0FF204610BD34
:1081700038B508460D4600F012FF04462146284651
:10818000FEF7E4FF204638BD7047FFFF044B002296
:108190001A714FF47A711A73024A99601A60704723
:1081A000A891FF1FD0BE000008B5034B01221A6042
:1081B000024B1B68984708BD0C710340C091FF1F1C
:1081C00008B5034B01221A60024B5B68984708BD53
:1081D0001C710340C091FF1F08B5034B01221A60B8
:1081E000024B9B68984708BD2C710340C091FF1F4C
:1081F00008B5034B01221A60024BDB68984708BDA3
:108200003C710340C091FF1F054B1A6842F4000205
:108210001A60044B00221A60034B01221A70704747
:108220003C80044000700340BC91FF1F064B0122BC
:108230001A6003F588333C331A6822F400021A608E
:10824000024B00221A70704700700340BC91FF1F60
:10825000F0B54578134C144F2B011A194260134A9C
:108260009E188660066947F8256000259D501951C3
:10827000032199504378427B4433DBB2037303F10B
:10828000604303F5644301211A70027B53119B0084
:1082900003F1604303F5614302F01F0201FA02F2A9
:1082A0001A60F0BD00710340C091FF1F08710340C8
:1082B000F8B50C4B1B7806460F460BB9FFF7A4FF29
:1082C0000024094D625DE3B23AB930467370394615
:1082D000FFF7BEFF01202855F8BD0134042CF0D172
:1082E0000020F8BDBC91FF1FB891FF1F82680023DA
:1082F00010B51360027B0121541102F01F0201FA34
:1083000002F2084941F82420074A41785354D15CCD
:1083100031B90133042BFAD1BDE81040FFF786BF15
:1083200010BD00BF80E100E0B891FF1F037870B579
:1083300004460D4616461BB1FFF7D8FF00232370F5
:10834000256120463146FFF7B3FF10B101232370AA
:1083500000E02070207870BD037810B504460BB1A2
:10836000FFF7C4FF0023237010BD08B5F8F77AF8B3
:10837000F8F7E2F900F014F9FAE700F0EFBC00F0CA
:10838000F5BC2DE9F04100258C688AB00746884687
:108390002E4694B12B46404601A9212200F0E7F871
:1083A0003B68202C34BF224620225B68384601A956
:1083B0001544A41A98470644EBE730460AB0BDE8D6
:1083C000F081FFFF07B5064B1B88ADF8043003684A
:1083D00001A95B680222984703B05DF804FB00BF67
:1083E00020BF000008B503685B689847002008BDFF
:1083F0000EB403B503AA52F8041B019200F0C0FEAC
:1084000002B05DF804EB03B0704770B505468AB062
:1084100022B90368C9B21B6898472CE0012A08BF3B
:108420000A2221B930228DF82520212413E02124AD
:10843000B1FBF2F002FB1011C9B209290AAE94BFD8
:10844000303137312644C9B206F8241C014610B138
:10845000013CE4B2ECE733B1013CE4B20AAB2344A3
:108460002D2203F8242C2B6801A95B68284621449F
:10847000C4F1220298470AB070BD0029BABF494230
:108480002D2300230A22FFF7C0BFFFF733BCFFF7FD
:10849000EFBBFFF713BCFFF7AFBC0846FFF7A0BC6C
:1084A00008461146FFF734BC7047FFFF044B00221B
:1084B0001A714FF47A711A73024A99601A60704700
:1084C000D091FF1F30BF000010B50446006800F0D7
:1084D0004DFC204610BD38B504460D4600680131FC
:1084E00000F024FD10B184E82100012038BD43686C
:1084F0008B4210B5044606D2FFF7EDFF20B1A3680A
:108500000BB922681370012010BDF8B504460F4660
:10851000154622B9036803B11A7000230BE0114617
:10852000FFF7E5FF064640B9206810B100F01EFCD9
:10853000266000236360A36004E0A56020683946DC
:1085400000F025FD2046F8BD38B500230446036041
:108550004360836003730D4639B1084600F01FFD88
:10856000294602462046FFF7D0FF204638BD38B5E1
:108570000C469AB191B181688B4202D300232370DB
:1085800038BDC91A551E8D4228BF0D4601682A46BE
:108590001944204600F022FD0023635538BDFFFF3B
:1085A00010B50E4C2378BBB901232370FFF7A2FB53
:1085B00008B1FFF779FFFEF78FF808B1FFF7E0FC8D
:1085C000FEF76CFB08B1FFF75DFDFEF7E7FD08B1B4
:1085D000FFF7DAFD0023237010BD00BFE091FF1FFD
:1085E00010B50023B0FBF2F402FB1400092894BF7D
:1085F00030303730C0B2C85420460CB10133F1E7F7
:10860000CA18547022469A4206DA885CCC5C8C54B4
:10861000C8540132013BF6E7084610BD1FB572B6DB
:10862000154B70221A70154A412111700F2102F862
:10863000011C80221A701A781206FCD5104B18689B
:1086400062B6104B984298BF0A2301AC98BF5843BA
:1086500021460A22FFF7C4FF0023E15C0A4A29B140
:1086600002EB430001330A2B4180F6D101335B005A
:10867000137004B010BD00BF0000024007000240AC
:10868000080002407F9698000088FF1F80F000409D
:1086900002E000BF81F0004142001FBF5FEA4103DA
:1086A00092EA030F7FEA226C7FEA236C6AD04FEADA
:1086B0001262D2EB1363C1BFD2184140484041401F
:1086C000B8BF5B42192B88BF704710F0004F40F4D1
:1086D000000020F07F4018BF404211F0004F41F4ED
:1086E000000121F07F4118BF494292EA030F3FD0B9
:1086F000A2F1010241FA03FC10EB0C00C3F12003CC
:1087000001FA03F100F0004302D5494260EB40005A
:10871000B0F5000F13D3B0F1807F06D340084FEAC5
:10872000310102F10102FE2A51D2B1F1004F40EBBA
:10873000C25008BF20F0010040EA03007047490022
:1087400040EB000010F4000FA2F10102EDD1B0FAED
:1087500080FCACF1080CB2EB0C0200FA0CF0AABFE2
:1087600000EBC25052421843BCBFD0401843704780
:1087700092F0000F81F4000106BF80F40000013286
:10878000013BB5E74FEA41037FEA226C18BF7FEA5D
:10879000236C21D092EA030F04D092F0000F08BF9F
:1087A0000846704790EA010F1CBF0020704712F086
:1087B0007F4F04D1400028BF40F00040704712F1C5
:1087C00000723CBF00F50000704700F0004343F02A
:1087D000FE4040F4000070477FEA226216BF084660
:1087E0007FEA23630146420206BF5FEA412390EA23
:1087F000010F40F4800070474FF0000304E000BF19
:1088000010F0004348BF40425FEA000C08BF7047C9
:1088100043F0964301464FF000001CE050EA01028D
:1088200008BF70474FF000030AE000BF50EA0102A2
:1088300008BF704711F0004302D5404261EB41018F
:108840005FEA010C02BF84460146002043F0B643B4
:1088500008BFA3F18053A3F50003BCFA8CF2083AD9
:10886000A3EBC25310DB01FA02FC634400FA02FCE2
:10887000C2F12002BCF1004F20FA02F243EB0200E9
:1088800008BF20F00100704702F1200201FA02FC4B
:10889000C2F1200250EA4C0021FA02F243EB02003E
:1088A00008BF20EADC7070474FF0FF0C1CEAD05282
:1088B0001EBF1CEAD15392EA0C0F93EA0C0F6FD043
:1088C0001A4480EA010C400218BF5FEA41211ED021
:1088D0004FF0006343EA501043EA5111A0FB01310D
:1088E0000CF00040B1F5000F3EBF490041EAD371E2
:1088F0005B0040EA010062F17F02FD2A1DD8B3F15E
:10890000004F40EBC25008BF20F00100704790F0CC
:10891000000F0CF0004C08BF49024CEA502040EA1E
:1089200051207F3AC2BFD2F1FF0340EAC2507047E4
:1089300040F400004FF00003013A5DDC12F1190F22
:10894000DCBF00F000407047C2F10002410021FA94
:1089500002F1C2F1200200FA02FC5FEA310040F1AC
:10896000000053EA4C0308BF20EADC70704792F025
:10897000000F00F0004C02BF400010F4000F013A5D
:10898000F9D040EA0C0093F0000F01F0004C02BF58
:10899000490011F4000F013BF9D041EA0C018FE7C7
:1089A0000CEAD15392EA0C0F18BF93EA0C0F0AD0CD
:1089B00030F0004C18BF31F0004CD8D180EA0100F3
:1089C00000F00040704790F0000F17BF90F0004F8C
:1089D000084691F0000F91F0004F14D092EA0C0F6E
:1089E00001D142020FD193EA0C0F03D14B0218BF01
:1089F000084608D180EA010000F0004040F0FE4047
:108A000040F40000704740F0FE4040F440007047E2
:108A10004FF0FF0C1CEAD0521EBF1CEAD15392EA61
:108A20000C0F93EA0C0F69D0A2EB030280EA010C51
:108A300049024FEA402037D04FF0805343EA1111EA
:108A400043EA10130CF000408B4238BF5B0042F148
:108A50007D024FF4000C8B4224BF5B1A40EA0C00ED
:108A6000B3EB510F24BFA3EB510340EA5C00B3EB1F
:108A7000910F24BFA3EB910340EA9C00B3EBD10F0D
:108A800024BFA3EBD10340EADC001B0118BF5FEA5F
:108A90001C1CE0D1FD2A3FF650AF8B4240EBC25088
:108AA00008BF20F0010070470CF0004C4CEA502049
:108AB0007F32C2BFD2F1FF0340EAC250704740F498
:108AC00000004FF00003013A37E792F0000F00F08A
:108AD000004C02BF400010F4000F013AF9D040EA08
:108AE0000C0093F0000F01F0004C02BF490011F49C
:108AF000000F013BF9D041EA0C0195E70CEAD15394
:108B000092EA0C0F08D142027FF47DAF93EA0C0F7A
:108B10007FF470AF084676E793EA0C0F04D14B025E
:108B20003FF44CAF08466EE730F0004C18BF31F010
:108B3000004CCAD130F000427FF45CAF31F000430A
:108B40007FF43CAF5FE700BF4FF0FF3C06E000BFA3
:108B50004FF0010C02E000BF4FF0010C4DF804CDC6
:108B60004FEA40024FEA41037FEA226C18BF7FEAD6
:108B7000236C11D001B052EA530C18BF90EA010FD8
:108B800058BFB2EB030088BFC81738BF6FEAE17067
:108B900018BF40F0010070477FEA226C02D15FEA03
:108BA000402C05D17FEA236CE4D15FEA412CE1D06F
:108BB0005DF8040B704700BF844608466146FFE736
:108BC0000FB5FFF7C9FF002848BF10F1000F0FBD18
:108BD0004DF808EDFFF7F4FF0CBF012000205DF811
:108BE00008FB00BF4DF808EDFFF7EAFF34BF012096
:108BF00000205DF808FB00BF4DF808EDFFF7E0FF2F
:108C000094BF012000205DF808FB00BF4DF808ED7F
:108C1000FFF7D2FF94BF012000205DF808FB00BFE2
:108C20004DF808EDFFF7C8FF34BF012000205DF8C4
:108C300008FB00BF4FEA4002B2F1FE4F0FD34FF0E6
:108C40009E03B3EB12620DD94FEA002343F00043B9
:108C500010F0004F23FA02F018BF404270474FF067
:108C60000000704712F1610F01D1420205D110F0EE
:108C7000004008BF6FF0004070474FF000007047A1
:108C800042000ED2B2F1FE4F0BD34FF09E03B3EB76
:108C9000126209D44FEA002343F0004323FA02F0A2
:108CA00070474FF00000704712F1610F01D142028E
:108CB00002D14FF0FF3070474FF00000704700BF07
:108CC00003460846194600F013B800210A2200F0B6
:108CD00019BA00210A2200F015BAFFFF0A4603491B
:108CE00003460868194600F07BB800BF7888FF1F6C
:108CF00070B5064C06460D4613462CB131462A4641
:108D00000220AFF3008070BD204670BD000000005F
:108D100070B50E4B0E4DED1AAD1000241E46AC4240
:108D200004D056F8242090470134F8E703F008FAFD
:108D3000084D094BED1AAD1000241E46AC4204D07C
:108D400056F8242090470134F8E770BD4CC100006C
:108D50004CC1000064C100004CC10000024B014640
:108D6000186800F08FB800BF7888FF1F024B0146DB
:108D7000186800F043B800BF7888FF1F10B5C9B26B
:108D800002449042034606D01C788C4200F1010058
:108D9000F7D1184610BD002010BD814270B501D337
:108DA00000230EE08C18A042FAD28518134613F166
:108DB000FF3305D3514266182944F65CCE54F6E7DA
:108DC00070BD934203D0CC5CC4540133F9E770BD4D
:108DD00002440346934202D003F8011BFAE77047AE
:108DE00038B502FB01F4214600F04CF8054618B1F5
:108DF00000212246FFF7ECFF284638BD30B5002998
:108E00003CD051F8042C0B1F1D49002AB8BF9B18F9
:108E10000A680C4612B95A600B6030BD93420DD2FD
:108E200019685818904203D15A5811444268196081
:108E30005A60236030BD994203D80A465168002920
:108E4000F9D1146815199D420AD11B682344D01822
:108E50008842136012D10868034413604B680CE029
:108E600002D90C23036030BD18681C188C4203D152
:108E70000C684968204418605960536030BD00BFD9
:108E8000E891FF1F70B5CD1C25F0030508350C2DAA
:108E900038BF0C25002D06463FDB8D423DD3214BCC
:108EA0001C6818462146A1B10B685B1B0ED40B2B26
:108EB00003D90B60CC18CD501FE08C4202D1626800
:108EC00002601AE04B6863600C4616E00C46496885
:108ED000E9E7154C23681BB9304600F031F82060F3
:108EE0002946304600F02CF8431C014615D0C41C1E
:108EF00024F0030484420AD1256004F10B00231DF1
:108F000020F00700C31A0BD05A42E25070BD304621
:108F1000611A00F015F80130EED10C233360002007
:108F200070BD00BFE891FF1FE491FF1F0A4603498F
:108F300003460868194600F001BA00BF7888FF1F91
:108F400038B5064C0023054608462360FCF70CFEA6
:108F5000431C02D1236803B12B6038BD0492FF1F6C
:108F6000C9B2024610F8013B1BB18B42F9D1104641
:108F700070470029FBD01846704710F8012B11F8F4
:108F8000013B012A28BF9A42F7D0D01A7047034606
:108F900011F8012B03F8012B002AF9D17047034681
:108FA00013F8012B002AFBD1181A0138704770B54D
:108FB00092B10B4605461C7810F8016BB44201F1E2
:108FC000010101D1012A03D128781B78C01A70BD94
:108FD000013A002CEDD1F7E7104670BD10B50346FD
:108FE00032B111F8014B03F8014B013A002CF7D1D3
:108FF0001A44934203D0002103F8011BF9E710BD86
:1090000084463F482DE9F04FD0F800800E463446A4
:1090100014F8015B08EB0500407800F0080000F050
:10902000FF0708B12646F2E72D2D03D1B41C757851
:10903000012703E02B2D04BF7578B41C33F010001A
:109040000DD1302D08D1207800F0DF00582851D103
:1090500065781023023402E0002B08BF0A23002F9A
:109060000CBF6FF0004A4FF0004ABAFBF3F900263C
:1090700003FB19AA304608EB050B9BF801B01BF067
:10908000040F01D0303D0BE01BF0030B1BD0BBF1F4
:10909000010F14BF4FF0570B4FF0370BCBEB05050B
:1090A0009D4210DAB6F1FF3F0AD0484506D801D1FB
:1090B000554503DC03FB0050012601E04FF0FF366D
:1090C00014F8015BD7E7731C0CD1002F4FF022037B
:1090D0000CBF6FF000404FF00040CCF800302AB9D0
:1090E000BDE8F08F07B1404242B106B1611E116088
:1090F000BDE8F08F002B08BF0823B0E7BDE8F08F74
:109100007C88FF1F30B51346044A05460C4610689C
:1091100029462246BDE83040FFF772BF7888FF1F1E
:109120002DE9F041ADF5047D1D464FF400730F4667
:1091300090460393044618B183690BB900F094F884
:1091400004AE00952046314603AA434600F05FF97D
:10915000054670B1204639462A46039B00F01EF8AA
:10916000B542039003D020462946FFF747FE0398F7
:1091700001E04FF0FF300DF5047DBDE8F081FFFF09
:1091800030B51346044A05460C4610682946224667
:10919000BDE83040FFF7C4BF7888FF1F38B5074CE3
:1091A000054600202060084611461A46FFF71AF9C6
:1091B000431C02D1236803B12B6038BD0492FF1F0A
:1091C000F8B5074600F1480494B1A5686668013E09
:1091D0000CD4AB89012B07D9B5F90E30013303D07C
:1091E0003846294600F0D6F96835F0E72468EBE701
:1091F000F8BDFFFF002310B50446036043608360A1
:1092000081814366C28103614361836119465C3099
:109210000822FFF7DDFD054B6362054BA362054B9A
:10922000E362054B2462236310BD00BF89930000F5
:10923000AB930000E39300000794000070B54B1E51
:1092400068255D430E4605F17401FFF71BFE0446D9
:1092500040B1002180E842000C30A06005F16802B6
:10926000FFF7B6FD204670BD836910B5044633BBD9
:109270008364C3640365124B124A1B68826298427E
:1092800004BF0123836100F01FF86060204600F0F6
:109290001BF8A060204600F017F80421E0600022CF
:1092A0006068FFF7A7FFA06809210122FFF7A2FF6E
:1092B000E06812210222FFF79DFF0123A36110BD88
:1092C000A4BF0000C1910000F8B51B4B1E68B36934
:1092D000074613B93046FFF7C7FF4836B4687368CE
:1092E000013B04D4B4F90C5075B16834F8E7336825
:1092F0002BB938460421FFF7A1FF306008B136686A
:10930000ECE70C233B60F8BD4FF6FF73E3810123CC
:10931000A38165662560A560656025616561A561BD
:1093200004F15C0029460822FFF752FD6563A5633E
:10933000A564E5642046F8BDA4BF0000F8B5064664
:1093400014460D4621B91146BDE8F840FFF79ABD15
:109350001AB9FFF753FD2046F8BD00F057F9A042B7
:109360000ED230462146FFF78DFD074650B1294603
:109370002246FCF741F830462946FFF73FFD01E061
:109380002846F8BD3846F8BD10B50C46B1F90E10A8
:1093900000F046F9002803DB636D0344636510BDEC
:1093A000A38923F48053A38110BD2DE9F0411D460C
:1093B0008B89DB0507460C46164605D5B1F90E101C
:1093C0000022022300F010F9A389B4F90E1023F44F
:1093D0008053A381384632462B46BDE8F041FFF763
:1093E000DDBE10B50C46B1F90E1000F0FDF8431CBF
:1093F000A38903D123F48053A38110BD43F4805388
:10940000A381606510BDB1F90E1000F02FB830B522
:1094100015469BB0146829B124B14FF4C162ADF870
:109420000C2005E04FF422720024ADF80C202146F8
:10943000002C0091049103DA8B230360002012E0DA
:109440004FF6FF72ADF80E2069461A461E9B029435
:10945000059400F053F9031E4FF0000003DB2B606E
:10946000009B187004981BB030BDFFFF38B5064C48
:109470000023054608462360FCF780FB431C02D10D
:10948000236803B12B6038BD0492FF1F8A892DE940
:10949000F041054610070C4657D44B68002B02DC00
:1094A0000B6C002B18DDE66AB6B102F48052002383
:1094B00092B22F682B600AB1626D10E0216A2846D3
:1094C0000123B047411C024609D12B683BB11D2B3B
:1094D00001D0162B46D12F600020BDE8F081A38972
:1094E0005B0705D56368D21A636B0BB1236CD21A84
:1094F000E66A216A28460023B047461CA28905D1A6
:109500002B681BB11D2B01D0162B19D100236360D2
:10951000D1042369236004D5421C01D12B6803B90F
:109520006065616B2F600029D6D004F14403994235
:1095300002D02846FFF762FC00206063BDE8F0819E
:1095400042F04002A281BDE8F0810E69002EC3D036
:109550000B680E60C6EB030893070CBF4B69002332
:109560008B6012E0A38943F04003A3814FF0FF30EA
:10957000BDE8F081A76A216A284632464346B847CB
:109580000028EFDD0644C0EB0808B8F1000FF1DC5D
:10959000A2E7FFFF38B50B6905460C46DBB118B1F1
:1095A00083690BB9FFF760FE0C4B9C4201D16C68DC
:1095B00008E00B4B9C4201D1AC6803E0094B9C4294
:1095C00008BFEC68B4F90C302BB128462146BDE841
:1095D0003840FFF75BBF002038BD00BFACC00000C3
:1095E000CCC00000ECC0000038B5074C0546002098
:1095F0002060084611461A46FCF7C3FA431C02D104
:10960000236803B12B6038BD0492FF1F51F8040C8E
:10961000002802DA04390B58184404387047FFFF59
:1096200038B5074C054600202060084611461A460A
:10963000FCF7A2FA431C02D1236803B12B6038BDAA
:109640000492FF1F2DE9F0478D68AB4281460C461E
:1096500092461F4643D38B8913F4906F3DD0266802
:109660000969C1EB06086669022206EB460696FB0D
:10967000F2F608F101023A44964238BF16465B05FD
:109680000FD53146FFF7FEFB054698B121694246EA
:10969000FBF7B2FEA38923F4906343F08003A38118
:1096A00013E03246FFF74AFE054670B94846216985
:1096B000FFF7A4FB0C23C9F80030A38943F0400353
:1096C000A3814FF0FF30BDE8F08725616661454416
:1096D000C8EB06062560A6603D46AF4200D23D4677
:1096E0002A4620685146FFF758FBA3685B1BA3601E
:1096F00023681D4425600020BDE8F0872DE9F04374
:109700009DB0074603938B891C060D4616460CD563
:109710000B6953B94021FFF7B5FB2860286110B9E8
:109720000C233B60C8E040236B6100230993202396
:109730008DF8293030238DF82A3033461C4613F833
:10974000012B1AB9B4EB06090FD002E0252AF5D196
:10975000F8E73846294632464B46FFF773FF01309B
:1097600000F0A580099B4B4409932378002B00F05F
:109770009E8000234FF0FF320493079305920693D7
:109780008DF853301A9304F101094C464D4E21785F
:1097900030460522FFF7F2FA09F10109049B28B1CE
:1097A000861B0120B04003430493EEE7D90644BF73
:1097B00020228DF853201A0744BF2B228DF8532006
:1097C00022782A2A02D0079B21460EE0039A111D17
:1097D00012680391002A01DB079204E0524243F031
:1097E00002030792049301340AE00C460131227807
:1097F000303A092A03D80A2000FB0323F5E7079330
:1098000023782E2B1AD163782A2B0AD1039B1A1D99
:109810001B680392002B04F10204B8BF4FF0FF3322
:109820000BE0611C00230C4601312278303A092AF2
:1098300003D80A2000FB0323F5E70593224E217885
:1098400030460322FFF79AFA30B1861B049B402072
:10985000B04003430493013421781C488DF828104C
:109860000622661CFFF78AFA88B1194B33B9039BAD
:10987000073323F007030833039314E003AB00938B
:10988000384604A92A46134BAFF3008007E003AB28
:109890000093384604A92A460E4B00F08FF8B0F129
:1098A000FF3F804603D0099B4344099345E7AB89BA
:1098B0005B0601D4099801E04FF0FF301DB0BDE810
:1098C000F08300BF0CC1000012C1000016C10000EF
:1098D00000000000459600002DE9F84315461F469C
:1098E0008A680B69DDF820809A42A8BF13462B6076
:1098F00091F8432006460C460AB101332B602368D9
:10990000990602D52B6802332B60236813F00609F1
:109910001DD094F843302268003318BF012392060B
:109920001FD5E1185A1C302081F84300224494F8D6
:10993000451082F84310023313E03046394604F1F3
:1099400019020123C047013007D009F10109E2687B
:109950002B68D31A9945F0DBDBE74FF0FF30BDE809
:10996000F8833046394604F14302C0470130F4D051
:1099700023682A68E16803F00603042B08BFC2EBE2
:1099800001052369A2680CBF25EAE57500259A4206
:10999000C4BFC3EB0203ED184FF00009A9450ADA72
:1099A0003046394604F11A020123C0470130D4D0B1
:1099B00009F10109F2E70020BDE8F8832DE9FF472E
:1099C0000E7E0C9D6E2E80460C4691469A4601F105
:1099D000430000F0A58011D8632E22D009D8002EB4
:1099E00000F0AF80582E40F0BF8081F845607B4A80
:1099F0004FE0642E1ED0692E1CD0B5E0732E00F00F
:109A0000A48009D86F2E2BD0702E40F0AD800B684B
:109A100043F020030B6038E0752E21D0782E34D02F
:109A2000A2E02B681A1D1B682A6001F1420781F829
:109A300042309DE022682B6812F0800F03D01A1D7F
:109A40002A601D6805E05106F9D51A1D2A60B3F990
:109A50000050002D39DA2D236D4284F8433034E074
:109A600022682B6812F0800F03D01A1D2A601D682F
:109A700004E05206F9D51A1D2A601D88237E574A34
:109A80006F2B14BF0A2308231BE07823544A84F861
:109A900045302368296813F0800F01F104062E6019
:109AA00001D00D6802E05F06FBD50D88DE0744BFDC
:109AB00043F0200323601DB9236823F020032360B3
:109AC0001023002184F8431001E0444A0A23666809
:109AD000A660002E03DB216821F00401216005B996
:109AE0006EB104F14201B5FBF3F603FB16550F46C8
:109AF000555D01F801593546002EF4D100E00746C6
:109B0000082B0AD12368DD0707D5626823699A42CA
:109B100003DC302307F8013C013FC01B20612CE02F
:109B200009682B68626911F0800F04D0191D296043
:109B30001B681A6005E04906F8D5191D29601B68E5
:109B40001A8000232361074617E02B681A1D2A603C
:109B50001F683846FFF723FA63682061984288BF80
:109B600023612369636005E004F1420784F84260E1
:109B700001232361002384F84330CDF800A0404640
:109B8000214603AA4B46FFF7A7FE013002D14FF052
:109B9000FF301FE0404649463A462369D04701302E
:109BA000F5D023689B0705D4E068039B9842B8BFB3
:109BB00018460FE00025E268039BD31A9D42F3DAB2
:109BC0004046494604F119020123D0470130DED056
:109BD0000135F0E704B0BDE8F08700BF1DC100000B
:109BE0002EC10000436F6E6E656374656420746FF0
:109BF0002045524F5320626F6172642061742025AA
:109C0000646270732E20426F617264204657207622
:109C1000657273696F6E2025642E0A0A4272696448
:109C20006765206D6F646520656E61626C65642098
:109C3000666F7220496E7465726E616C2044657641
:109C400069636520626F6F746C6F61646572206117
:109C500063636573732E0A57616974696E67206662
:109C60006F7220746865206669727374206368611E
:109C700072616374657220746F20726573657420FD
:109C800074686520696E7465726E616C20505355FE
:109C90002E2E2E2E005B4254204E4F542050524503
:109CA00053454E545D0041542B554152543D25645B
:109CB0002C302C30000D0A004F4B00415400415411
:109CC0002B4E414D453F0041542B505357443F00CC
:109CD0005B4D41494E4252445F554E53555052548C
:109CE00045445D0041542B4E414D453D2573004197
:109CF000542B505357443D2530346900636C735FD7
:109D0000436972634275666665725F3100636C73A6
:109D1000436972634275666665725F320044756DB1
:109D200070696E672043697263756C617220627539
:109D3000666665725F006275666665725F2073694C
:109D40007A652069733A2025640A00252E3278202E
:109D500000FFFFFFFFFFFFFF00000000000000000A
:109D6000895B00002915000041150000000000007B
:109D70001801FFFFFFFFFFFF0000000000000000D0
:109D800069150000351500005515000000000000A1
:109D90005B74696D656F75745D0A005B25645D2099
:109DA0005B25645D0A005B706172616D735F636F58
:109DB000756E742025645D205B25645D0A00556E18
:109DC0006B6E6F776E20737461746520696E2063AB
:109DD000616C6C6261636B20696E20636C73436FAE
:109DE0006E736F6C652121210A00496E69742064CD
:109DF000796E207061636B65740050617274696C78
:109E00006C79206F70656E2068616E642066756E77
:109E10006374696F6E616C697479206973206E6F09
:109E2000742079657420696D706C656D656E7465FC
:109E30006420696E2074686973206669726D776149
:109E400072652076657273696F6E2E20504C656165
:109E50007365207573652074686520636F6D6D612F
:109E60006E6420746F2073657420736572766F2042
:109E7000706F736974696F6E7320696E6469766957
:109E80006475616C6C792E0A00436C6F7365206891
:109E9000616E642066756E6374696F6E616C69745F
:109EA00079206973206E6F742079657420696D70F4
:109EB0006C656D656E74656420696E207468697385
:109EC0002076657273696F6E2E20557365207468F5
:109ED0006520636F6D6D616E6420746F20736574AF
:109EE00020736572766F20706F736974696F6E731B
:109EF00020696E646976696475616C6C792E0A00FC
:109F00005363616E6E696E6720696E2070726F6751
:109F10007265732E2055736520636F6D6D616E647D
:109F200020277374617475732720746F206C6973B4
:109F3000742049447320666F756E642E00596573F2
:109F4000004E6F005365656420526F626F746963E1
:109F5000732045524F53204669726D776172650ACE
:109F6000004669726D776172652076657273696FFC
:109F70006E2025642C20636F6D70696C6564206FA2
:109F80006E204A756E20203920323031372031372B
:109F90003A35373A303700202853455249414C3141
:109FA0005F4F4E455F5749524520646566696E654F
:109FB00064290A000A426F617264206D6F64656CE7
:109FC0002025640A00426F61726420485720436F65
:109FD0006E66696775726174696F6E2025640A0028
:109FE00053657269616C204E756D62657220252E15
:109FF0003278252E3278252E32780A004375727217
:10A00000656E742073656E736F7220726573697309
:10A01000746F722076616C75653A2025640A00427F
:10A020006F61726420697320636F6E666967757211
:10A03000656420746F206F70657261746520776944
:10A040007468203132626974207265736F6C757444
:10A05000696F6E2E0A00426F61726420697320631B
:10A060006F6E6669677572656420746F206F7065C6
:10A070007261746520776974682031306269742078
:10A080007265736F6C7574696F6E2E0A000A45787D
:10A090007465726E616C2062757320636F6D6D758F
:10A0A0006E69636174696F6E2073657474696E673D
:10A0B000733A200A00426F617264206275732064F3
:10A0C00065766963652049443A2025640A00526533
:10A0D0007475726E2064656C61792074696D653A7F
:10A0E000202564205B2564206D6963726F7365634E
:10A0F000735D0A00537461747573207265747572B0
:10A100006E206C6576656C3A2025640A005573698B
:10A110006E6720545820456E61626C652070696ED0
:10A120003A2025730A000A496E7465726E616C20CC
:10A1300062757320636F6D6D756E69636174696FAD
:10A140006E2073657474696E67733A20000A496EF5
:10A150007465726E616C2062757320426175642053
:10A16000726174652073657474696E673A20256442
:10A17000203D202564204250530A000A4120426CB1
:10A180007565746F6F746820636F6D6D756E69634C
:10A190006174696F6E206D6F64756C6520697320E2
:10A1A00070726573656E743A0A00426C7565746FFF
:10A1B0006F746820434F4D4D204261756420736574
:10A1C0007474696E67202564203D20256420425008
:10A1D000530A00426C7565746F6F7468206465760D
:10A1E000696365206E616D653A202573200A00421F
:10A1F0006C7565746F6F746820646576696365203B
:10A20000636F64653A2025303464200A000A4E6F7B
:10A2100020426C7565746F6F746820636F6D6D7527
:10A220006E69636174696F6E206D6F64756C652013
:10A2300064657465637465642E0A004F6E004F6632
:10A240006600426F617264205374617475733A0AD8
:10A2500000496E7465726E616C2054656D70657234
:10A2600061747572653A09256420646567430A0064
:10A2700045787465726E616C20537570706C7920CE
:10A28000566F6C746167653A0925642E2564560A19
:10A2900000436F6E6669677572656420566F6C74F3
:10A2A00061676520696E20496E7465726E616C200D
:10A2B0004275733A092564560A0A00506F7369742F
:10A2C000696F6E2053656E736F72205741646475B9
:10A2D0006374696F6E3A0925640A00506F7369747C
:10A2E000696F6E2053656E736F722057466C657888
:10A2F000696F6E3A0925640A0050616C6D204F70D9
:10A30000746963616C2053656E736F7220696E733C
:10A3100074616C6C65643A0925730A0050616C6D58
:10A32000204F70746963616C2053656E736F722087
:10A33000416D6269656E74204C696768743A0925DD
:10A34000640A0050616C6D204F70746963616C2009
:10A3500053656E736F7220436F6D70757465642002
:10A3600052656164696E673A0925640A0043617049
:10A37000616369746976652053656E736F727320CB
:10A38000696E7374616C6C65643A0925730A0043E5
:10A390006170616369746976652053656E736F726D
:10A3A00020312072656164696E673A0925640A008C
:10A3B000436170616369746976652053656E736F7C
:10A3C0007220322072656164696E673A0925640AF9
:10A3D000000A436F6D6D756E69636174696F6E20FD
:10A3E000537461746973746963733A0A0055415216
:10A3F000543120284578742E436F6D6D29204275A5
:10A4000066666572204F76657272756E733A2025A6
:10A41000640A0055415254322028496E742E436F0D
:10A420006D6D2920427566666572204F7665727281
:10A43000756E733A2025640A005541525433205BEF
:10A4400042542E436F6D6D5D2042756666657220C5
:10A450004F76657272756E733A2025640A000A534E
:10A460006572766F2049447320286C6973743A20B2
:10A4700049442C205B4552524F52204D41534B5D75
:10A48000290A002564095B4D41494E424F4152441F
:10A490005D0A002564095B25645D0A000A506F723D
:10A4A00074207374617475733A0A00506F7274206B
:10A4B00025642043757272656E742052656164690B
:10A4C0006E673A204F5645524C4F414420455252F8
:10A4D0004F52202825646D41290A00506F72742064
:10A4E00025642043757272656E74205265616469DB
:10A4F0006E673A2025646D410A000A4120426C755E
:10A5000065746F6F746820636F6D6D756E696361DC
:10A5100074696F6E206D6F64756C6520697320704F
:10A52000726573656E742E0A00426C7565746F6F88
:10A53000746820706F776572207374617475733AF4
:10A540002025730A005365656420526F626F746939
:10A5500063732045524F53204669726D776172656F
:10A560002C2076657273696F6E2025640A0A004C90
:10A57000697374206F6620616476616E6365642020
:10A58000636F6D6D616E64732E0A5741524E494E72
:10A59000473A20546865736520636F6D6D616E6422
:10A5A00073206172652072657365727665642066DA
:10A5B0006F722074686520757365206F662053651F
:10A5C000656420526F626F74696373207465636899
:10A5D0006E6963616C206167656E74732E0A496EE3
:10A5E000636F7272656374207573616765206D6156
:10A5F0007920636175736520696E6F70657261742F
:10A60000696F6E2C2064616D61676520616E6420E6
:10A610006D617920766F696420796F75722077613A
:10A620007272616E74792E0A557365206174207997
:10A630006F7572206F776E207269736B2E0A0A0035
:10A640006168700954686973206D6573736167652B
:10A650002E0A00696E697420656570726F6D0A005C
:10A66000696E697420626F6172646D6F64656C20DD
:10A670005B6D6F64656C5D0A00696E697420626F62
:10A680006172646877636F6E666967205B636F6E83
:10A69000666967206D61736B5D0A00696E6974207D
:10A6A00063757272656E747265736973746F72200C
:10A6B0005B7265736973746F722076616C75652067
:10A6C0004F686D735D0A00696E697420736E205B5C
:10A6D00059595D205B4D4D5D205B434845434B53CD
:10A6E000554D5D0A00696E69742073657269616C0D
:10A6F000636F6D6D205B6C6566747C7269676874EE
:10A700005D0A0A005573652027636F6E66696727C7
:10A7100020666F72207468652072656D61696E696C
:10A720006E6720636F6E66696775726174696F6EBC
:10A73000732E2054797065202768656C7027206619
:10A740006F7220696E666F726D6174696F6E2E0A2A
:10A750000A005365656420526F626F7469637320E9
:10A7600045524F53204669726D7761726520766558
:10A770007273696F6E2025640A0A004C6973742035
:10A780006F6620617661696C61626C6520636F6DD4
:10A790006D616E64732E20416C6C20636F6D6D6112
:10A7A0006E64732061726520636173652073656EEA
:10A7B0007369746976652E0A0A0068656C700954BD
:10A7C000686973206D6573736167652E0A00737421
:10A7D0006174757309446973706C61792063757273
:10A7E00072656E742073797374656D20737461740F
:10A7F00075732E0A0061626F757409446973706C19
:10A80000617920696E7465726E616C20696E666F25
:10A81000726D6174696F6E2E0A007363616E62758A
:10A82000730952657363616E732074686520696E85
:10A830007465726E616C2062757320666F7220445D
:10A84000796E616D6978656C20646576696365739E
:10A850002E0A00736574706F73205B64657669639C
:10A86000652069645D205B706F736974696F6E3A0F
:10A8700020302D25645D0953657420706F736974F1
:10A88000696F6E20666F72207370656369666965B3
:10A8900064206465766963652E0A0072657374616D
:10A8A0007274205B7073757C616C6C5D09526573AA
:10A8B0007461727473206F6E6C7920746865207394
:10A8C0006572766F20505355206F72207468652032
:10A8D00066756C6C2073797374656D2E0A00636FF6
:10A8E0006E666967205B657874626175647C657803
:10A8F0007469647C6578747478656E61626C657C7B
:10A9000031326269746164636578706F7365647C09
:10A91000696E74626175647C6274626175647C6284
:10A92000746E616D657C6274636F64657C62746370
:10A930006F6D6D616E645D205B76616C75655D0A3F
:10A940000953797374656D207769646520636F6E50
:10A9500066696775726174696F6E206F7074696F74
:10A960006E732E0A00636F6D6D6272696467652095
:10A970005B6269746D61736B5D09456E61626C65E4
:10A9800020434F4D4D206272696467652E0A09426B
:10A9900069746D61736B3A20313D5553422C2032FE
:10A9A0003D496E74204275732C20343D45787420E7
:10A9B0004275732C20383D42542C2031363D55537E
:10A9C0004220772F4454522052657365742E0A003A
:10A9D000777262205B6465766963652069645D20D7
:10A9E0005B616464726573735D205B62797465207A
:10A9F00076616C75655D095772697465206279745A
:10AA00006520746F206465766963652E0A0077722D
:10AA100077205B6465766963652069645D205B61AE
:10AA20006464726573735D205B696E742076616C1B
:10AA300075655D09577269746520776F726420745B
:10AA40006F206465766963652E0A00726562205B1B
:10AA50006465766963652069645D205B6164647226
:10AA60006573735D0952656164206279746520665F
:10AA7000726F6D206465766963652E0A0072657772
:10AA8000205B6465766963652069645D205B616451
:10AA900064726573735D095265616420776F7264D7
:10AAA0002066726F6D206465766963652E0A0A0000
:10AAB000496E76616C696420636F6D6D616E642EA2
:10AAC00020436F6D6D616E647320617265206361F8
:10AAD00073652073656E7369746976652E0A54799F
:10AAE0007065202768656C702720666F72206D6F17
:10AAF000726520696E666F726D6174696F6E2E0A81
:10AB0000004944206E6F742070726573656E742006
:10AB1000696E2074686520696E7465726E616C2060
:10AB20006275732E20547970652027737461747573
:10AB3000732720666F722061206C697374206F66C2
:10AB40002076616C6964204944732E0A00496E7650
:10AB5000616C696420706F736974696F6E2E204D2B
:10AB60006178696D756D20616363657074656420DB
:10AB7000706F736974696F6E206973203430393572
:10AB80002E0A41637475616C206D6178696D756D15
:10AB900020646570656E6473206F6E2061637475E8
:10ABA00061746F7220636F6E666967757261746934
:10ABB0006F6E2E0A0070737500446F6E6500616CD5
:10ABC0006C00506172616D657465722070617373A1
:10ABD00065642028222573222920697320696E76F6
:10ABE000616C69642E204269746D61736B206D75B0
:10ABF0007374207365742074776F20696E74657246
:10AC000066616365732E0A00446F6E652E00657879
:10AC1000747478656E61626C6500796573006E6F3F
:10AC20000031326269746164636578706F73656462
:10AC300000696E74626175640062746261756400BB
:10AC4000496E76616C69642073657474696E672EF1
:10AC50002053657474696E672073686F756C642027
:10AC600062652061204261756420706172616D656A
:10AC700074657220286578616D706C653A20313694
:10AC80003D31313532303062707329005375636560
:10AC9000737320636F6E6669677572696E672042B1
:10ACA00054206D6F64756C652E0A004661696C6591
:10ACB0006420636F6E6669677572696E67204254BF
:10ACC000206D6F64756C652E0A0053617665642093
:10ACD00073657474696E6720696E204D61696E20BA
:10ACE000626F61726420656570726F6D2E006274B0
:10ACF0006E616D65005375636573730A0046616923
:10AD00006C0A006274636F646500496E76616C69F9
:10AD10006420636F64652E20436F6465206D7573D6
:10AD20007420626520612034206469676974206E34
:10AD3000756D6572696320636F64652072616E670B
:10AD4000696E672066726F6D203030303020746F0E
:10AD500020393939392E0A00537563636573732EB0
:10AD600020425420636F64652073657420746F20E3
:10AD7000272573272028616C77617973206120343F
:10AD800020646967697420636F6465292E0A006214
:10AD900074636F6D6D616E64005265706C793A0A10
:10ADA00025730A00656570726F6D00626F61726471
:10ADB0006D6F64656C00626F6172646877636F6E5B
:10ADC0006669670063757272656E74726573697324
:10ADD000746F720073657269616C636F6D6D006C86
:10ADE00065667400726967687400736E0068656CEC
:10ADF0007000616870007374617475730061626FD4
:10AE00007574007363616E62757300636C6F736554
:10AE100000706172746F70656E00736574706F732B
:10AE2000007265737461727400636F6D6D62726934
:10AE300064676500777262007772770072656200FE
:10AE400072657700466978656453697A6544786C01
:10AE5000436F6D6D616E6451756575650046697807
:10AE6000656453697A6544786C436F6D6D616E6497
:10AE700051756575655F6279746573617272617928
:10AE800000466978656453697A6544786C436F6DF0
:10AE90006D616E6451756575655F62696469726C38
:10AEA000697374000A44554D50204C4953540A00AC
:10AEB0004865616420616464722025702C205461AF
:10AEC000696C20616464722025702C204974656D62
:10AED00020636F756E742025642C2070747220645A
:10AEE00069666572656E63652025640A0041646465
:10AEF000722025702C20536572766F2049442025DE
:10AF0000640A00636C735F4D61696E426F617264C5
:10AF10005F696E697400FFFF000000000000000020
:10AF2000DD400000E9390000193A0000000000008F
:10AF3000736C6176657061727365723A696E7420C4
:10AF400064657669636573206461746100FFFFFF67
:10AF500000000000000000002144000065410000E6
:10AF60008D4100009F410000ED410000394200008A
:10AF700081420000CB4500007D470000000000003A
:10AF80000000000000000000895B00009D490000F7
:10AF9000C5490000895B0000895B0000895B0000F7
:10AFA000895B0000895B0000895B000000000000F5
:10AFB000000000000100000002000000030000008B
:10AFC0000400000006000000070000000800000068
:10AFD000090000000A0000000B0000000C00000047
:10AFE0000D0000000E0000000F0000001000000027
:10AFF0001100000012000000130000001400000007
:10B0000015000000160000001800000019000000E4
:10B010001A0000001B0000001C0000001D000000C2
:10B020001E0000001F0000002000000021000000A2
:10B030002200000023000000240000002500000082
:10B040002600000027000000280000002900000062
:10B050002A0000002B0000002C0000002D00000042
:10B060002E0000002F000000300000003100000022
:10B070003200000033000000340000003500000002
:10B0800036000000370000003800000039000000E2
:10B090003A0000003B0000003C0000003D000000C2
:10B0A0003E0000003F0000004000000041000000A2
:10B0B0004200000043000000440000004400000083
:10B0C0004500000046000000470000004800000066
:10B0D000490000004A0000004B0000004C00000046
:10B0E0004D0000004E0000004F0000005000000026
:10B0F0005100000052000000530000005400000006
:10B1000055000000560000005700000058000000E5
:10B1100058000000590000005A0000005B000000C9
:10B120005C0000005D0000005E0000005F000000A9
:10B130006000000061000000620000006300000089
:10B14000640000006500000066000000660000006A
:10B150006700000068000000690000006A0000004D
:10B160006B0000006C0000006D0000006E0000002D
:10B170006F0000007000000071000000720000000D
:10B1800072000000730000007400000075000000F1
:10B1900076000000770000007800000079000000D1
:10B1A0007A0000007B0000007C0000007C000000B2
:10B1B0007D0000007E0000007F0000008000000095
:10B1C0008100000082000000830000008400000075
:10B1D0008500000086000000860000008700000057
:10B1E00088000000890000008A0000008B00000039
:10B1F0008C0000008D0000008E0000008F00000019
:10B200008F000000900000009100000092000000FC
:10B2100093000000940000009500000096000000DC
:10B2200097000000970000009800000099000000BF
:10B230009A0000009B0000009C0000009D000000A0
:10B240009E0000009F0000009F000000A000000082
:10B25000A1000000A2000000A3000000A400000064
:10B26000A5000000A6000000A7000000A700000045
:10B27000A8000000A9000000AA000000AB00000028
:10B28000AC000000AD000000AE000000AF00000008
:10B29000AF000000B0000000B1000000B2000000EC
:10B2A000B3000000B4000000B5000000B6000000CC
:10B2B000B6000000B7000000B8000000B9000000B0
:10B2C000BA000000BB000000BC000000BD00000090
:10B2D000BE000000BE000000BF000000C000000073
:10B2E000C1000000C2000000C3000000C400000054
:10B2F000C5000000C5000000C6000000C700000037
:10B30000C8000000C9000000CA000000CB00000017
:10B31000CC000000CD000000CD000000CE000000F9
:10B32000CF000000D0000000D1000000D2000000DB
:10B33000D3000000D4000000D4000000D5000000BD
:10B34000D6000000D7000000D8000000D90000009F
:10B35000DA000000DB000000DC000000DC00000080
:10B36000DD000000DE000000DF000000E000000063
:10B37000E1000000E2000000E3000000E400000043
:10B38000E4000000E5000000E6000000E700000027
:10B39000E8000000E9000000EA000000EB00000007
:10B3A000EB000000EC000000ED000000EE000000EB
:10B3B000EF000000F0000000F1000000F2000000CB
:10B3C000F3000000F3000000F4000000F5000000AE
:10B3D000F6000000F7000000F8000000F90000008F
:10B3E000FA000000FB000000FC000000FC00000070
:10B3F000FD000000FE000000FF0000000001000052
:10B40000010100000201000003010000040100002E
:10B410000401000005010000060100000701000012
:10B4200008010000090100000A0100000B010000F2
:10B430000C0100000D0100000D0100000E010000D4
:10B440000F010000100100001101000012010000B6
:10B450001301000014010000150100001601000096
:10B460001701000017010000180100001901000079
:10B470001A0100001B0100001C0100001D0100005A
:10B480001E0100001F01000020010000210100003A
:10B49000210100002201000023010000240100001E
:10B4A00025010000260100002701000028010000FE
:10B4B000290100002A0100002B0100002C010000DE
:10B4C0002D0100002D0100002E0100002F010000C1
:10B4D00030010000310100003201000033010000A2
:10B4E0003401000035010000360100003701000082
:10B4F00038010000390100003A0100003B01000062
:10B500003B0100003C0100003D0100003E01000045
:10B510003F01000040010000410100004201000025
:10B520004301000044010000450100004601000005
:10B530004701000048010000490100004A010000E5
:10B540004B0100004C0100004D0100004E010000C5
:10B550004F0100004F0100005001000051010000A8
:10B560005201000053010000540100005501000089
:10B570005601000057010000580100005901000069
:10B580005A0100005B0100005C0100005D01000049
:10B590005E0100005F010000600100006101000029
:10B5A0006201000063010000640100006501000009
:10B5B00066010000670100006801000069010000E9
:10B5C0006A0100006B0100006C0100006D010000C9
:10B5D0006E0100006F0100007001000071010000A9
:10B5E0007201000073010000740100007501000089
:10B5F0007601000077010000780100007901000069
:10B600007A0100007B0100007C0100007D01000048
:10B610007E0100007F010000800100008101000028
:10B620008201000083010000840100008501000008
:10B630008601000088010000890100008A010000E5
:10B640008B0100008C0100008D0100008E010000C4
:10B650008F010000900100009101000092010000A4
:10B660009301000094010000950100009601000084
:10B6700097010000980100009A0100009B01000062
:10B680009C0100009D0100009E0100009F01000040
:10B69000A0010000A1010000A2010000A301000020
:10B6A000A4010000A6010000A7010000A8010000FD
:10B6B000A9010000AA010000AB010000AC010000DC
:10B6C000AD010000AE010000B0010000B1010000BA
:10B6D000B2010000B3010000B4010000B501000098
:10B6E000B6010000B7010000B9010000BA01000076
:10B6F000BB010000BC010000BD010000BE01000054
:10B70000C0010000C1010000C2010000C30100002F
:10B71000C4010000C5010000C7010000C80100000D
:10B72000C9010000CA010000CB010000CC010000EB
:10B73000CE010000CF010000D0010000D1010000C7
:10B74000D2010000D4010000D5010000D6010000A4
:10B75000D7010000D8010000DA010000DB01000081
:10B76000DC010000DD010000DF010000E00100005D
:10B77000E1010000E2010000E4010000E501000039
:10B78000E6010000E7010000E9010000EA01000015
:10B79000EB010000EC010000EE010000EF010000F1
:10B7A000F0010000F2010000F3010000F4010000CC
:10B7B000F5010000F7010000F8010000F9010000A8
:10B7C000FB010000FC010000FD010000FF01000082
:10B7D0000002000001020000030200000402000059
:10B7E0000502000007020000080200000902000034
:10B7F0000B0200000C0200000D0200000F0200000E
:10B8000010020000120200001302000014020000E7
:10B810001602000017020000190200001A020000C0
:10B820001B0200001D0200001E020000200200009A
:10B830002102000023020000240200002602000072
:10B8400027020000280200002A0200002B0200004C
:10B850002D0200002E020000300200003102000024
:10B8600033020000340200003602000037020000FC
:10B87000390200003A0200003C0200003E020000D3
:10B880003F020000410200004202000044020000AA
:10B890004502000047020000490200004A02000081
:10B8A0004C0200004D0200004F0200005102000057
:10B8B000520200005402000056020000570200002D
:10B8C000590200005B0200005C0200005E02000002
:10B8D00060020000610200006302000065020000D7
:10B8E00066020000680200006A0200006C020000AC
:10B8F0006D0200006F020000710200007302000080
:10B900007402000076020000780200007A02000053
:10B910007C0200007E0200007F0200008102000025
:10B9200083020000850200008702000089020000F7
:10B930008B0200008D0200008E02000090020000C9
:10B94000920200009402000096020000980200009B
:10B950009A0200009C0200009E020000A00200006B
:10B96000A2020000A4020000A6020000A80200003B
:10B97000AB020000AD020000AF020000B102000007
:10B98000B3020000B5020000B7020000B9020000D7
:10B99000BC020000BE020000C0020000C2020000A3
:10B9A000C4020000C7020000C9020000CB02000070
:10B9B000CE020000D0020000D2020000D50200003A
:10B9C000D7020000D9020000DC020000DE02000005
:10B9D000E1020000E3020000E5020000E8020000CE
:10B9E000EA020000ED020000F0020000F202000096
:10B9F000F5020000F7020000FA020000FC0200005D
:10BA0000FF0200000203000005030000070300001E
:10BA10000A0300000D0300001003000012030000E1
:10BA200015030000180300001B0300001E030000A4
:10BA30002103000024030000270300002A03000064
:10BA40002D03000030030000330300003603000024
:10BA5000390300003D0300004003000043030000E1
:10BA6000460300004A0300004D030000500300009D
:10BA700054030000570300005B0300005E03000056
:10BA80006203000065030000690300006D0300000D
:10BA90007103000074030000780300007C030000C1
:10BAA0008003000084030000880300008C03000072
:10BAB0009003000094030000980300009D03000021
:10BAC000A1030000A5030000AA030000AE030000CC
:10BAD000B3030000B8030000BC030000C103000072
:10BAE000C6030000CB030000D0030000D503000014
:10BAF000DA030000DF030000E5030000EA030000B2
:10BB0000EF030000F5030000FB0300000004000049
:10BB1000060400000C0400001204000019040000D8
:10BB20001F040000250400002C0400003304000062
:10BB30003A04000040040000480400004F040000E4
:10BB4000560400005E040000660400006E0400005D
:10BB5000760400007E0400008704000090040000CA
:10BB600099040000A2040000AC040000B604000028
:10BB7000C0040000CA040000D5040000E004000076
:10BB8000EC040000F80400000405000011050000AA
:10BB90001E0500002C0500003A05000049050000C4
:10BBA00059050000690500007A0500008C050000B9
:10BBB0009F050000B3050000C8050000DE05000079
:10BBC0004D616C6C6F63206661696C656420666FA3
:10BBD000722025730A005061636B65743A2000304F
:10BBE0007846462030784646203078004545505209
:10BBF0004F4D2077726974652064656E69656420B5
:10BC0000627920696E7465726E616C2070726F74F7
:10BC1000656374696F6E2E204E72206F6620777296
:10BC20006974657320617474656D707465642069EE
:10BC30006E20746869732073657373696F6E3A2040
:10BC400000417474656D7074696E6720746F20773D
:10BC500072697465206120424954206F6E20612012
:10BC60006269746D61702062757420697427732035
:10BC70006F7574206F662072616E67653B20746813
:10BC80006520616C6C6F7765642072616E676520FA
:10BC9000697320307E372E00090AFFFFFFFFFFFF88
:10BCA000FFFFFFFFFFFFFF0D00060807FFFF0E0F5E
:10BCB000FF0CFFFFFFFFFFFF0B05050E08090D0C32
:10BCC00006070F04001303931A9217C5858486870D
:10BCD000C4FF6FF07F030370037813F0800FFBD075
:10BCE0007047FFFF4008FE4340A004404408FE4365
:10BCF00044A004400018FE4300C004403000FE434E
:10BD0000309004403400FE43349004401C18FE433D
:10BD10001CC004401018FE4310C004400818FE4325
:10BD200008C004400C18FE430CC004400C10FE4335
:10BD30000CB004401010FE4310B004401810FE4335
:10BD400018B004401C10FE431CB004401410FE4305
:10BD500014B004400418FE4304C004400010FE4325
:10BD600000B004400008FE4300A004400408FE4365
:10BD700004A004400C08FE430CA004400808FE4345
:10BD800008A004401418FE4314C004401818FE43D1
:10BD900018C004400410FE4304B004400810FE43E1
:10BDA00008B004401400FE43149004404C08FE43C5
:10BDB0004CA004400420FE4304D004402410FE4361
:10BDC00024B004402010FE4320B004402810FE435D
:10BDD00028B004402C10FE432CB004400020FE4349
:10BDE00000D004404808FE4348A004401000FE4331
:10BDF00010900440090AFFFFFFFFFFFFFFFFFFFF56
:10BE0000FFFFFF0D00060807FFFF0E0FFF0CFFFFEF
:10BE1000FFFFFFFF0B05FFFF000000000000000018
:10BE2000417F0000597F0000297F0000317F000022
:10BE30002D7F0000357F0000CD7E0000DF7E0000FA
:10BE4000FF7E0000037F0000097F0000197F0000D3
:10BE5000397F00003D7F00009D7E0000A97E00002C
:10BE6000B57E0000C17E0000697F00004D7F0000AC
:10BE70000000000000000000458000005D80000020
:10BE80002D800000358000003180000039800000E6
:10BE9000D17F0000E37F00000380000007800000E6
:10BEA0000D8000001D8000003D80000041800000EA
:10BEB000A17F0000AD7F0000B97F0000C57F0000BA
:10BEC0006D800000518000000000000000000000B4
:10BED000498100006181000031810000398100004A
:10BEE000358100003D810000D5800000E780000022
:10BEF000078100000B8100001181000021810000FA
:10BF00004181000045810000A5800000B180000053
:10BF1000BD800000C98000007181000055810000D3
:10BF20000D0AFFFFFFFFFFFF000000000000000000
:10BF30009B840000A18400008B8400008F8400009B
:10BF4000938400009784000000151915000100007B
:10BF50007887FF1F1200000000020000A287FF1F69
:10BF60004300000000030000FC87FF1F00000000EA
:10BF7000010309048A87FF1F00000000020309046F
:10BF8000E687FF1F00000000030309040088FF1F6D
:10BF900000000000000000000000000000000000A1
:10BFA0004300FFFF1888FF1F0020202020202020B2
:10BFB0002020282828282820202020202020202059
:10BFC0002020202020202020208810101010101069
:10BFD00010101010101010101004040404040404B5
:10BFE000040404101010101010104141414141414F
:10BFF0000101010101010101010101010101010131
:10C000000101010110101010101042424242424240
:10C010000202020202020202020202020202020200
:10C0200002020202101010102000000000000000A8
:10C030000000000000000000000000000000000000
:10C0400000000000000000000000000000000000F0
:10C0500000000000000000000000000000000000E0
:10C0600000000000000000000000000000000000D0
:10C0700000000000000000000000000000000000C0
:10C0800000000000000000000000000000000000B0
:10C0900000000000000000000000000000000000A0
:10C0A000000000000000000000FFFFFF0000000093
:10C0B0000000000000000000000000000000000080
:10C0C0000000000000000000000000000000000070
:10C0D0000000000000000000000000000000000060
:10C0E0000000000000000000000000000000000050
:10C0F0000000000000000000000000000000000040
:10C10000000000000000000000000000232D302B84
:10C110002000686C4C006566674546470030313248
:10C12000333435363738394142434445460030319F
:10C13000323334353637383961626364656600FFFF
:10C14000F8B500BFF8BC08BC9E4670473504000037
:10C15000C5500000857F0000898000008D810000AF
:04C16000AD840000AA
:10C1640000000000010000000A0400000892FF1F04
:10C1740008000000FFFFFFFF120100020200004060
:10C18400C016830400010102030118035400650072
:10C1940065006E00730079006400750069006E002C
:10C1A4006F0009024300020100C0320904000001CB
:10C1B40002020100052400100105240101010424E8
:10C1C4000206052406000107058203100040090445
:10C1D4000100020A000000070503024000000705F1
:10C1E4008402400000001603550053004200200062
:10C1F400530065007200690061006C0004030904C7
:10C204000C0300000000000000000000000000001B
:10C21400000000000000000000000000ACC00000AE
:10C22400CCC00000ECC000000000000000000000D2
:10C234000000000000000000A0BF0000000000009B
:10C2440000000000000000000000000000000000EA
:10C2540000000000000000000000000000000000DA
:10C2640000000000000000000000000000000000CA
:10C2740000000000000000001888FF1FA8BF000095
:00000001FF
